:100000000C94A5150C941A160C941A160C941A1626
:100010000C941A160C941A160C941A160C941A16A0
:100020000C941A160C941A160C941A160C941A1690
:100030000C941A160C9482180C94C2180C941A166C
:100040000C941A160C941A160C941A160C941A1670
:100050000C941A160C941A160C941A160C941A1660
:100060000C941A160C941A160C941A160C941A1650
:100070008100450027FF24FF2A902B1C210C22FB26
:10008000850084008903888D81096F0244424700FE
:100090004501B083B300B10125118A4F8B035A5536
:1000A00001200101003808000000000000000000ED
:1000B00000000000000000000000000000004C1BD9
:1000C0004F1BAD1BB21BBA1B581B5D1B621BC31B16
:1000D000651B681B6B1BA71BAA1BD31B00408891C9
:1000E000D2E4ADB5B6BEBFFF505245535320535472
:1000F00041525400494E5345525420434F494E00FB
:10010000435245444954533A0000000000000000A7
:1001100000000000000000000000000000000000DF
:1001200000000000000000000000000000000000CF
:1001300000000000000000000000000000000000BF
:100140000000000000000000000000FFFFFF0000B2
:10015000000000FFFFFF0000000000FFFFFF0000A5
:10016000000000FFFF000000000000FFFF00000093
:100170000000000000000000000000FFFF00000081
:100180000000000000000000000000FF00FF000071
:10019000000000FF00FF0000000000FF00FF000063
:1001A000000000000000000000000000000000004F
:1001B000000000000000000000000000000000003F
:1001C00000000000000000000000FF000000FF0031
:1001D00000FFFFFFFFFFFFFF0000FF000000FF0028
:1001E0000000FF000000FF000000FF000000FF0013
:1001F00000FFFFFFFFFFFFFF0000FF000000FF0008
:10020000000000000000000000000000FF000000EF
:100210000000FFFFFFFFFFFF00FF0000FF000000E6
:100220000000FFFFFFFFFF0000000000FF0000FFD5
:1002300000FFFFFFFFFFFF0000000000FF000000C5
:10024000000000000000000000FFFF0000000000B0
:1002500000FFFF0000FF000000000000FF000000A2
:10026000000000FF000000000000FF000000000090
:1002700000FF0000FFFF000000000000FFFF000083
:100280000000000000000000000000FFFF00000070
:100290000000FF0000FF00000000FFFF00FF000063
:1002A0000000FFFFFF00000000FF0000FFFF00FF55
:1002B00000FF000000FFFF000000FFFFFFFF00FF46
:1002C00000000000000000000000FFFF0000000030
:1002D0000000FFFF00000000000000FF0000000021
:1002E0000000FF000000000000000000000000000F
:1002F00000000000000000000000000000000000FE
:1003000000000000000000000000000000FFFF00EF
:1003100000000000FF000000000000FF00000000DF
:10032000000000FF00000000000000FF00000000CF
:1003300000000000FF0000000000000000FFFF00C0
:100340000000000000000000000000FFFF000000AF
:100350000000000000FF0000000000000000FF009F
:10036000000000000000FF00000000000000FF008F
:100370000000000000FF0000000000FFFF00000080
:10038000000000000000000000000000000000006D
:1003900000000000FF0000000000FF00FF00FF0061
:1003A000000000FFFFFF00000000FF00FF00FF0053
:1003B00000000000FF00000000000000000000003E
:1003C000000000000000000000000000000000002D
:1003D00000000000FF00000000000000FF0000001F
:1003E0000000FFFFFFFFFF0000000000FF00000013
:1003F00000000000FF0000000000000000000000FE
:1004000000000000000000000000000000000000EC
:1004100000000000000000000000000000000000DC
:100420000000000000000000000000FFFF000000CE
:10043000000000FFFF0000000000FFFF00000000C0
:1004400000000000000000000000000000000000AC
:10045000000000000000000000000000000000009C
:100460000000FFFFFFFFFF00000000000000000091
:10047000000000000000000000000000000000007C
:10048000000000000000000000000000000000006C
:10049000000000000000000000000000000000005C
:1004A000000000000000000000000000000000004C
:1004B000000000FFFF000000000000FFFF00000040
:1004C000000000000000000000000000000000FF2D
:1004D000000000000000FF000000000000FF00001E
:1004E00000000000FF000000000000FF000000000E
:1004F0000000FF000000000000FF000000000000FE
:100500000000000000000000000000FFFFFF0000EE
:100510000000FF0000FFFF0000FFFF000000FFFFE2
:1005200000FFFF000000FFFF00FFFF000000FFFFD3
:100530000000FFFF0000FF00000000FFFFFF0000C1
:10054000000000000000000000000000FFFF0000AD
:10055000000000FFFFFF000000000000FFFF0000A0
:1005600000000000FFFF000000000000FFFF00008F
:1005700000000000FFFF00000000FFFFFFFFFFFF83
:1005800000000000000000000000FFFFFFFFFF0070
:1005900000FFFF000000FFFF0000000000FFFFFF62
:1005A000000000FFFFFFFF000000FFFFFFFF000053
:1005B00000FFFFFF0000000000FFFFFFFFFFFFFF45
:1005C00000000000000000000000FFFFFFFFFFFF31
:1005D0000000000000FFFF0000000000FFFF00001F
:1005E000000000FFFFFFFF00000000000000FFFF11
:1005F00000FFFF000000FFFF0000FFFFFFFFFF0004
:10060000000000000000000000000000FFFFFF00ED
:10061000000000FFFFFFFF000000FFFF00FFFF00E2
:1006200000FFFF0000FFFF0000FFFFFFFFFFFFFFD5
:100630000000000000FFFF000000000000FFFF00BE
:10064000000000000000000000FFFFFFFFFFFF00B0
:1006500000FFFF000000000000FFFFFFFFFFFF00A2
:10066000000000000000FFFF000000000000FFFF8E
:1006700000FFFF000000FFFF0000FFFFFFFFFF0083
:100680000000000000000000000000FFFFFFFF006E
:100690000000FFFF0000000000FFFF00000000005E
:1006A00000FFFFFFFFFFFF0000FFFF000000FFFF54
:1006B00000FFFF000000FFFF0000FFFFFFFFFF0043
:1006C000000000000000000000FFFFFFFFFFFFFF31
:1006D00000FFFF000000FFFF0000000000FFFF0020
:1006E00000000000FFFF0000000000FFFF0000000E
:1006F000000000FFFF000000000000FFFF000000FE
:1007000000000000000000000000FFFFFFFF0000ED
:1007100000FFFF000000FF0000FFFFFF0000FF00E0
:100720000000FFFFFFFF000000FF0000FFFFFFFFD2
:1007300000FF00000000FFFF0000FFFFFFFFFF00C1
:1007400000000000000000000000FFFFFFFFFF00AE
:1007500000FFFF000000FFFF00FFFF000000FFFFA1
:100760000000FFFFFFFFFFFF000000000000FFFF91
:100770000000000000FFFF000000FFFFFFFF00007F
:100780000000000000000000000000000000000069
:10079000000000FFFF000000000000FFFF0000005D
:1007A0000000000000000000000000FFFF0000004B
:1007B000000000FFFF00000000000000000000003B
:1007C0000000000000000000000000000000000029
:1007D000000000FFFF000000000000FFFF0000001D
:1007E0000000000000000000000000FFFF0000000B
:1007F000000000FFFF0000000000FFFF00000000FD
:1008000000000000000000000000000000FF0000E9
:1008100000000000FF000000000000FF00000000DA
:100820000000FF0000000000000000FF00000000CA
:1008300000000000FF0000000000000000FF0000BA
:1008400000000000000000000000000000000000A8
:1008500000000000000000000000FFFFFFFFFF009D
:1008600000000000000000000000FFFFFFFFFF008D
:100870000000000000000000000000000000000078
:100880000000000000000000000000FF0000000069
:1008900000000000FF0000000000000000FF00005A
:1008A000000000000000FF000000000000FF00004A
:1008B00000000000FF000000000000FF000000003A
:1008C00000000000000000000000FFFFFFFFFF002D
:1008D00000FFFFFFFFFFFFFF00FFFF000000FFFF23
:1008E0000000000000FFFF00000000FFFFFF00000D
:1008F0000000000000000000000000FFFFFF0000FB
:100900000000000000000000000000FFFFFF0000EA
:100910000000FF000000FF0000FF0000FF00FF00DC
:1009200000FF00FF00FFFF0000FF0000FFFF0000CE
:100930000000FF0000000000000000FFFFFFFF00BC
:100940000000000000000000000000FFFFFF0000AA
:100950000000FFFF00FFFF0000FFFF000000FFFF9F
:1009600000FFFF000000FFFF00FFFFFFFFFFFFFF92
:1009700000FFFF000000FFFF00FFFF000000FFFF7F
:10098000000000000000000000FFFFFFFFFFFF006D
:1009900000FFFF000000FFFF00FFFF000000FFFF5F
:1009A00000FFFFFFFFFFFF0000FFFF000000FFFF51
:1009B00000FFFF000000FFFF00FFFFFFFFFFFF0041
:1009C0000000000000000000000000FFFFFFFF002B
:1009D0000000FFFF0000FFFF00FFFF00000000001D
:1009E00000FFFF000000000000FFFF00000000000B
:1009F0000000FFFF0000FFFF000000FFFFFFFF00FF
:100A0000000000000000000000FFFFFFFFFF0000EB
:100A100000FFFF0000FFFF0000FFFF000000FFFFDE
:100A200000FFFF000000FFFF00FFFF000000FFFFCE
:100A300000FFFF0000FFFF0000FFFFFFFFFF0000BF
:100A4000000000000000000000FFFFFFFFFFFFFFAD
:100A500000FFFF000000000000FFFF00000000009A
:100A600000FFFFFFFFFFFF0000FFFF00000000008E
:100A700000FFFF000000000000FFFFFFFFFFFFFF7F
:100A8000000000000000000000FFFFFFFFFFFFFF6D
:100A900000FFFF000000000000FFFF00000000005A
:100AA00000FFFFFFFFFFFF0000FFFF00000000004E
:100AB00000FFFF000000000000FFFF00000000003A
:100AC0000000000000000000000000FFFFFFFFFF2B
:100AD0000000FFFF0000000000FFFF00000000001A
:100AE00000FFFF0000FFFFFF00FFFF000000FFFF0F
:100AF0000000FFFF0000FFFF000000FFFFFFFFFFFF
:100B0000000000000000000000FFFF000000FFFFE9
:100B100000FFFF000000FFFF00FFFF000000FFFFDD
:100B200000FFFFFFFFFFFFFF00FFFF000000FFFFD0
:100B300000FFFF000000FFFF00FFFF000000FFFFBD
:100B400000000000000000000000FFFFFFFFFFFFAB
:100B500000000000FFFF000000000000FFFF000099
:100B600000000000FFFF000000000000FFFF000089
:100B700000000000FFFF00000000FFFFFFFFFFFF7D
:100B8000000000000000000000000000FFFFFFFF69
:100B90000000000000FFFF000000000000FFFF0059
:100BA0000000000000FFFF000000000000FFFF0049
:100BB00000FF000000FFFF000000FFFFFFFF00003C
:100BC000000000000000000000FFFF000000FFFF29
:100BD00000FFFF0000FFFF0000FFFF00FFFF00001D
:100BE00000FFFFFFFF00000000FFFFFFFFFF00000E
:100BF00000FFFF00FFFFFF0000FFFF0000FFFFFFFF
:100C000000000000000000000000FFFF00000000E6
:100C10000000FFFF000000000000FFFF00000000D8
:100C20000000FFFF000000000000FFFF00000000C8
:100C30000000FFFF000000000000FFFFFFFFFFFFBC
:100C4000000000000000000000FFFF000000FFFFA8
:100C500000FFFFFF00FFFFFF00FFFFFFFFFFFFFFA1
:100C600000FFFFFFFFFFFFFF00FFFF00FF00FFFF90
:100C700000FFFF000000FFFF00FFFF000000FFFF7C
:100C8000000000000000000000FFFF000000FFFF68
:100C900000FFFFFF0000FFFF00FFFFFFFF00FFFF5F
:100CA00000FFFFFFFFFFFFFF00FFFF00FFFFFFFF51
:100CB00000FFFF0000FFFFFF00FFFF000000FFFF3D
:100CC00000000000000000000000FFFFFFFFFF0029
:100CD00000FFFF000000FFFF00FFFF000000FFFF1C
:100CE00000FFFF000000FFFF00FFFF000000FFFF0C
:100CF00000FFFF000000FFFF0000FFFFFFFFFF00FD
:100D0000000000000000000000FFFFFFFFFFFF00E9
:100D100000FFFF000000FFFF00FFFF000000FFFFDB
:100D200000FFFF000000FFFF00FFFFFFFFFFFF00CD
:100D300000FFFF000000000000FFFF0000000000B7
:100D400000000000000000000000FFFFFFFFFF00A8
:100D500000FFFF000000FFFF00FFFF000000FFFF9B
:100D600000FFFF000000FFFF00FFFF00FFFFFFFF8D
:100D700000FFFF0000FFFF000000FFFFFFFF00FF7C
:100D8000000000000000000000FFFFFFFFFFFF0069
:100D900000FFFF000000FFFF00FFFF000000FFFF5B
:100DA00000FFFF0000FFFFFF00FFFFFFFFFF00004D
:100DB00000FFFF00FFFFFF0000FFFF0000FFFFFF3D
:100DC00000000000000000000000FFFFFFFF000027
:100DD00000FFFF0000FFFF0000FFFF000000000019
:100DE0000000FFFFFFFFFF00000000000000FFFF0A
:100DF00000FFFF000000FFFF0000FFFFFFFFFF00FC
:100E000000000000000000000000FFFFFFFFFFFFE8
:100E100000000000FFFF000000000000FFFF0000D6
:100E200000000000FFFF000000000000FFFF0000C6
:100E300000000000FFFF000000000000FFFF0000B6
:100E4000000000000000000000FFFF000000FFFFA6
:100E500000FFFF000000FFFF00FFFF000000FFFF9A
:100E600000FFFF000000FFFF00FFFF000000FFFF8A
:100E700000FFFF000000FFFF0000FFFFFFFFFF007B
:100E8000000000000000000000FFFF000000FFFF66
:100E900000FFFF000000FFFF00FFFF000000FFFF5A
:100EA00000FFFFFF00FFFFFF0000FFFFFFFFFF004D
:100EB000000000FFFFFF000000000000FF00000036
:100EC000000000000000000000FFFF000000FFFF26
:100ED00000FFFF000000FFFF00FFFF00FF00FFFF1B
:100EE00000FFFFFFFFFFFFFF00FFFFFFFFFFFFFF10
:100EF00000FFFFFF00FFFFFF00FFFF000000FFFFFC
:100F0000000000000000000000FFFF000000FFFFE5
:100F100000FFFFFF00FFFFFF0000FFFFFFFFFF00DC
:100F2000000000FFFFFF00000000FFFFFFFFFF00C9
:100F300000FFFFFF00FFFFFF00FFFF000000FFFFBB
:100F400000000000000000000000FFFF0000FFFFA5
:100F50000000FFFF0000FFFF0000FFFF0000FFFF99
:100F6000000000FFFFFFFF0000000000FFFF000087
:100F700000000000FFFF000000000000FFFF000075
:100F8000000000000000000000FFFFFFFFFFFFFF68
:100F90000000000000FFFFFF00000000FFFFFF0057
:100FA000000000FFFFFF00000000FFFFFF00000047
:100FB00000FFFFFF0000000000FFFFFFFFFFFFFF3B
:100FC0000000000000000000000000FFFFFFFF0025
:100FD000000000FFFF000000000000FFFF00000015
:100FE000000000FFFF000000000000FFFF00000005
:100FF000000000FFFF000000000000FFFFFFFF00F7
:101000000000000000000000000000FFFFFFFF00E4
:101010000000FF00000000FF00FF0000FFFF0000D5
:10102000FFFF00FF00000000FFFF00FF00000000C6
:10103000FFFF0000FFFF0000FF00FF00000000FFB7
:10104000000000FFFFFFFF00000000FFFFFFFF00A8
:101050000000000000FFFF000000000000FFFF0094
:101060000000000000FFFF000000000000FFFF0084
:101070000000000000FFFF00000000FFFFFFFF0076
:101080000000000000000000000000FF0000000061
:101090000000FF00FF00000000FF000000FF000054
:1010A0000000000000000000000000000000000040
:1010B0000000000000000000000000000000000030
:1010C0000000000000000000000000000000000020
:1010D0000000000000000000000000000000000010
:1010E0000000000000000000000000000000000000
:1010F000000000000000000000FFFFFFFFFFFFFFF7
:10110000000000000000000000FEFEFEFEFEFEFEED
:10111000FEFEFEFEFE5CFEFEFEFEFEFE1237FEFE44
:10112000FEFEFE525B2D52FEFE52FFAD6436ADADAB
:101130005B52A452642553A4ADFEFEFEFEFE00FEEB
:10114000FEFEFEFEFEFEFEFEFEFEFEFEFEFEFEFEBF
:10115000FEFEFEFE13FEFEFEFEFEFEFE3712FE004B
:10116000FEFEFEFE6D6DADADFFFEFEA4AD255BADDA
:10117000A4FEFFFF5C240900FEFEAD5252FEFEFEFF
:10118000FEFEFEFEFEFEFEFEFEFEFEFEFEFEFEFE7F
:10119000FEFEFE00FEFEFEFEFEFEFE252400A4FF77
:1011A000FFFEFE092E6DA45B00FEFE00AD251C5364
:1011B000FEFEFEA4AD5C09FEFEFEFEFFA400FEFEE8
:1011C000FEFEFE52FEFEFEFEFEFEFEFEFEFEFE00E9
:1011D00000FEFEFEFEFEADFF00FE001209A4FFA40D
:1011E000FEFE002E2E6D5C53FEFEFEFE5B2424FEF2
:1011F000FEFEFEFEADA453FEFEFEFE00FFAD00FEB1
:10120000FEFEFEFEFF52FEFEFEFEFEFEFE5BA4FEA6
:10121000FEFEFEFE00FFADFEFEFEFE0052AD5200E1
:10122000FE0013366D2425FEFEFE092464641CFEB8
:10123000FEFEFEFE52AD52FEFEFEFEFE00FFA4FECE
:10124000FEFEFEFEFE5B52FEFEFEFEFEFF52FEFEB8
:10125000FEFEFE00FFADFEFEFEFEFEFEAD5B09FEE5
:10126000FEFEFE09642524FEFEFE5B3F24645C5204
:10127000FEFE0009FEADFF52FEFEFEFEFE00FFADCB
:10128000FEFEFEFEFEFE0000FEFEFEADFEFEFEFECB
:10129000FEFE00FF5B52FEFEFEFEFEADA41C09FE3C
:1012A000FEFEFE5264251301FEFEFE1B2E64A452B8
:1012B000FEFE002E1252ADFF5BFEFEFEFEFEFE5253
:1012C000FEFEFEFEFEFEFEFEFEFEFEFEFEFEFEFE3E
:1012D000FE00FF5252FEFEFEFE00FFFF5C2401FEF8
:1012E000FEFE00A464255B5BFEFEFE002D64ADFFE8
:1012F000FFFEFE1237000000FEFEFE0909FEFEFEA4
:10130000FEFEFEFEFEFEFEFEFEFEFEFEFEFEFEFEFD
:10131000FEFEFE00FEFEFEFEFEA4AD52251C52A403
:10132000525BFFAD2464ADFF5BFEFE526D64520064
:10133000FEFEFEFE3624FEFEFEFEFEFE1309FEFE4F
:10134000FEFEFEFEFEFEFEFEFEFEFEFEFE5BA4FEBA
:10135000FEFEFEFEFEFFADFEFEFEFEFE52AD5200A4
:10136000FEFE13376E2525FEFEFE0924646D240063
:10137000FEFEFEFE52AD5200FEFEFEFE00FFA4FE8B
:10138000FEFEFEFEFEA452FEFEFEFEFEFEFEFE0081
:10139000FEFEFEFEFEFEADFFFEFEFEFE01A5FF5BB5
:1013A000FE00132D6E6D24FEFEFE0A2E6D6D24FED2
:1013B000FEFEFEFE01A4FF52FEFEFEFEFE00ADFF9D
:1013C000FEFEFEFEFEFE0000FEFEFEFEFEFEFEFE39
:1013D000FEFEFEFEFEFEFEFEFEFEFE0001535BFF75
:1013E00052FE092E5CADFFAD00001C3F2E6D640067
:1013F00000FEFE010AA4FFFF00FEFE00010152FFF5
:1014000052FEFEFEFEFEFEFEFEFEFEFEFEFEFEFEA8
:10141000FEFEFE000000FEFEFEFEFE01010AFE00D2
:10142000FE0012375B5CADFF5B001C3F65ADFFFF4C
:10143000ADFEFE0A0A0B005200FEFE000000FEFE9A
:10144000FEFEFEFEFEFEFEFEFE52AD0000FEFEFEB5
:10145000FEFEADFF000000FEFE485BFFAD5B5200EC
:10146000FE52ADEBEAADADAD5B485BFFAD5B52004C
:10147000FEFEADFF000000FEFE52AD0000FEFEFECF
:10148000FEFEFEFEFEFEFEFEFE525B0000FEFEFEC7
:10149000FEFE5B5B0000FEFEFE0B525B5252000044
:1014A000FE00521515525252000A525B5252000071
:1014B000FEFE5B5B0000FEFEFE525B0000FEFEFED9
:1014C000FEFEFEFEFEFEFEFEFEFEFEFE005AFEFEDE
:1014D000FEFEFEFE5159FEFEFEFEFE10116C10FED9
:1014E000FE08201224751B181100235B766E5B2307
:1014F00009FE1B521C155B1B00FE0A000001000ABE
:10150000FEFE0000FEFEFE00FEFEFE09FEFEFEFEEA
:10151000FEFEFE515AFEFE08FEFEFE087511093A57
:10152000FEFEFE222D755B6C0908205B76260A12F2
:101530000900235B5C25095209FEFE1C52FEFEFEDB
:10154000FEFEFE0000FEFEFEFEFEFEFEFEFEFEFEB7
:10155000FEFE635100103108FEFE5162096319243A
:10156000FEFE0809366C5B1209FE081A6C2F145B2C
:101570000AFE311A5B1313FEFEFE0824125BFEFE08
:10158000FEFEFEFE090AFEFEFEFEFEFEFE0800FE58
:10159000FEFEFEFE082023FEFE095A091A5B641CAB
:1015A00000FE5A75766D5C5200FEFE086C2E1DFE24
:1015B000FEFEFE095B0A09FEFEFE083A6C1252FEB0
:1015C000FEFEFEFE090901FEFEFEFE0008FEFEFE16
:1015D000FEFEFE0028241C0AFEFEFE18125B5200CE
:1015E000FE085A64751D15FEFE5A596C75362500A5
:1015F000FEFEFE18125B5BFEFEFEFEFE216D1B0A68
:10160000FEFEFEFE1009FEFEFEFEFEFEFE0000FED9
:10161000FEFE083A2C1209FEFEFEFE115B0A09FED0
:10162000FEFEFE086C1E25FEFEFE506C76765D000A
:10163000FE085A091A5B5B6401FEFEFE08182D00C5
:10164000FEFEFEFEFE10FEFEFEFEFEFE000AFEFE9A
:10165000FEFEFE1B125BFEFEFEFE3122095C0AFE50
:10166000FEFE10646C271C520AFE110935750A5BD8
:1016700009FE51B412645B24FEFE5950081030116B
:10168000FEFEFEFEFEFE00FEFEFEFEFEFEFEFEFE78
:10169000FEFEFE6509FEFEFEFEFE1B645C140909EB
:1016A0000108325B252F0A0909FE081A75755B6D62
:1016B00009FEFE097509093A00FEFE5A5AFEFE1996
:1016C000FEFEFE5A00FEFEFEFEFEFEFEFEFEFEFEDC
:1016D000FEFE0909FE00FE0AFEFE125B14245B1BDF
:1016E000FEFE255B16375C6D090030097575122109
:1016F00010FE08211B6C21FEFEFEFEFE5A5AFEFE65
:10170000FEFEFEFE5A5AFEFEFEFEFEFE190900FE19
:10171000FEFEFEFE186D645C00FEFE0000AD5BFE8A
:10172000FE09596B357F2709FE09596C35761E096C
:10173000FEFEFEFE5B1A125C0AFEFE103A3B1B091F
:10174000FEFEFEFEFEFEFEFEFEFEFE000800FEFEAB
:10175000FEFEFEFE282C245C00FEFE191B5B52528E
:1017600000085A63756E1609FE09596C357F2F09FA
:10177000FEFEFE191B5B5B52FEFEFEFE18231C5C88
:1017800000FEFEFE100800FEFEFEFEFEFEFEFEFE59
:10179000FEFEFE11202009FEFEFEFE006B2A6E6595
:1017A0000A095A6376761E09FE08AB747E771E0915
:1017B000FEFEFE0000645BFEFEFEFE0010B6640A44
:1017C000FEFEFE0021090000FEFEFEFEFEFEFEFE05
:1017D000FEFEFE192C1301FEFEFEFEFE632A120918
:1017E00000095A63343325120908AB6C35771F0999
:1017F000FEFEFEFE00645BFEFEFEFE0011645C0069
:10180000FEFEFE00190900FEFEFEFE000900FEFEBF
:10181000FEFEFE086C645CFEFEFEFEFE525B09FEF0
:10182000FE095A632C2B1D090008AB6C323B2E1BA2
:101830000AFEFEFE525B09FEFEFEFE0863645CFECD
:10184000FEFEFE000800FEFEFEFEFE00110900FE88
:10185000FEFEFE001A645C00FEFEFEFE005B5BFE08
:10186000FE095A6C756F1600FE5AAB6C7E75255BCF
:1018700000FEFEFE2A3A1B0900FEFE19751300FE4B
:10188000FEFEFE00FEFEFEFEFEFEFE0000FE00FE70
:10189000FEFEFEFE091100FEFEFEFEFE091200FE27
:1018A000FEFEFE010D0503FEFEFEFE03170F0DFEFC
:1018B000FEFEFE020E0E0CFEFEFEFE000C0D02FEF3
:1018C000FEFEFEFE010A00FEFEFE00FE09FEFEFE1A
:1018D000FEFE000911FEFEFEFEFEFE001303FEFEEC
:1018E000FEFEFE020D0E04FEFEFEFE020E0F0E00B8
:1018F000FEFEFE010D0E0501FEFEFEFE020C0CFEBC
:10190000FEFEFEFEFE0001FEFEFEFEFEFEFEFEFEF2
:10191000FEFEFE09FEFEFEFEFEFE09190A0301FEA2
:10192000FEFEFE0A0D0E0DFEFEFEFE020E0F0E0363
:10193000FEFEFEFE040E050CFEFEFEFEFE02030A87
:10194000FEFEFEFEFEFEFEFEFEFEFEFEFEFEFEFEB7
:10195000FEFEFEFEFEFEFEFEFEFE09090B0301FE7C
:10196000FE09081305170E03FEFEFE020E0F0E0DF4
:1019700001FEFEFE030E0D0401FEFEFEFEFEFEFE57
:10198000FEFEFEFEFEFEFEFEFEFEFEFEFEFEFEFE77
:10199000FEFEFEFEFEFEFEFEFEFEFEFE0B0403014C
:1019A000FEFE110A0E0F0E0D09FE110A0E0F0E0D8E
:1019B00001FEFEFE03040301FEFEFEFEFEFEFEFE31
:1019C000FEFEFEFEFEFEFEFEFEFEFEFEFEFEFEFE37
:1019D000FEFEFEFEFEFE00FEFEFEFEFE030E0D0CF3
:1019E00001FEFE0B0E0F0E0C010908130E0F0E0365
:1019F000FEFE12090B0301FEFEFEFEFEFEFEFEFED3
:101A0000FEFEFEFEFEFEFEFEFEFEFEFEFEFEFEFEF6
:101A1000FEFEFEFEFE020B0AFEFEFEFE040E0503A7
:101A2000FEFEFE030E0F0E0BFEFEFE0B050E0DFE60
:101A3000FEFE09180B0301FEFEFEFE09FEFEFEFE81
:101A4000FEFEFE00FEFEFEFEFEFEFEFEFEFE00FEB2
:101A5000FEFEFEFE020C03FEFEFEFE010E0E0D005B
:101A6000FEFEFE03170F0EFEFEFEFE030E0E04FE2C
:101A7000FEFEFE000B0BFEFEFEFEFE0811FEFEFE4D
:101A8000FEFEFEFE09FEFEFEFEFEFEFE0901FEFE5D
:101A9000FEFEFE010D0D01FEFEFEFE030E0E03FE18
:101AA000FEFEFE040F0F04FEFEFEFE0B0E0E03FEF6
:101AB000FEFEFEFE0A0AFEFEFEFEFEFE1111FEFE08
:101AC000FEFEFEFEFEFEFEFEFEFEFEFEFEFEFEFE36
:101AD000FEFEFEFE020302FEFE09FE0A0E0F0E04CB
:101AE000FEFE195D0E0F0F0D0A09FE0A0E0F060C01
:101AF000FEFEFEFE020302FEFEFEFEFEFEFEFEFEF9
:101B0000FEFEFEFEFEFEFEFEFEFEFEFE000101FEED
:101B1000FEFEFE010D0E0D03FE09FE0C0E5FA5FE7E
:101B2000FEFE190B5CA35B130909FE0C0E5FAEFEF3
:101B3000FEFEFE010D0E0D03FEFEFEFE000101FE87
:101B4000FEFEFEFEFEFEFEFEFEFEFE010C0D01FE92
:101B5000FEFE000D0F0AFEFEFE09090DA5ADADFE4D
:101B6000FEFE190B5B5B5B130909090DAEADADFE03
:101B7000FEFEFE050F53FEFEFEFEFE010C0D02FEF4
:101B8000FEFEFEFEFEFEFEFEFEFE010D03FEFEFE5E
:101B9000FEFE0C0E0000FEFEFE090B0CADADAD000E
:101BA000FEFE125C5B5B5B1309120B0CADADAD006E
:101BB000FEFE030E0052FEFEFEFE010D03FEFEFEC3
:101BC000FEFEFEFE0200FEFEFEFEFEFE0402FEFE25
:101BD000FEFEFE07171704FEFE04071F272F1F0334
:101BE000FE051F271F2F1707020F27372F1F270755
:101BF00004020D27172F3717FEFE02071F27070FB6
:101C0000FEFEFE040F0502FEFEFEFEFEFEFEFEFED2
:101C1000FEFEFE020402FEFEFEFE020D0F0502FEA7
:101C2000FEFE061F1F1F0504FE040D1F1F171F04C5
:101C3000FEFE0127071F17FEFEFEFE040402FEFE45
:101C4000FEFEFEFEFEFEFEFEFEFEFE00090000FEA3
:101C5000FEFE000313120C02FE00050E0C130E0E06
:101C60000101045C5B5C5B540301ADAD5B64ADAD35
:101C700001FE52000A120052FEFEFEFE0112FEFE9E
:101C8000FEFEFEFE000AFEFEFEFE0000120000FE4A
:101C9000FEFE0009130E1703FE00040D130A030CC9
:101CA00001010F025C5BADAD000203FE5B135252FB
:101CB000FEFE52AD005C09FEFEFEFE00FE0912FEB5
:101CC000FEFEFEFEFEFE09FEFEFEFE09010201FE14
:101CD000FEFEFE120E0F0401FE0012120B52AD5B4F
:101CE000FE010D0B5C5B5B52FE010F52AD1309FE52
:101CF000FE000DADA4FE5C09FEFE025252FE001372
:101D0000FEFEFEFEFEFEFEFEFEFEFEFE0202FEFEEB
:101D1000FEFEFE0D0F545BFEFEFE120D01ADADFE8C
:101D2000FE1213135C5BFEFEFEFE050BAD5C64123F
:101D3000FEFE0E0CAD52FE0A09FE0204AD52FEFE7E
:101D4000FEFEFE00FEFEFEFEFEFEFE0102FEFEFEAA
:101D5000FEFE020E54AD00FEFEFE040EA4A4FEFE26
:101D6000FE09130B5B5B12120909120BAD5C0A0A28
:101D700001FE040EADA4FEFEFEFE020E54AD00FEFA
:101D8000FEFEFE010201FEFEFEFEFEFEFEFEFEFE69
:101D9000FEFE030BA452FEFEFEFE0E03AD52FE0934
:101DA00009010E02AD125C0AFE090B135C5CFEFE1B
:101DB000FEFE120C01FFADFEFEFEFE0D0F54A4FE52
:101DC000FEFEFEFE0203FEFEFEFEFEFEFEFEFEFE2A
:101DD000FEFE015B00FE0913FE0103AD52FE65012C
:101DE000FE020652A41301FEFE010E0A5CAD5B006A
:101DF000FEFE131B0A52ADA4FE00FE120E0F0402DB
:101E0000FEFEFE09010201FEFEFEFEFEFEFE00FEDB
:101E1000FEFEFEFEFE090AFEFEFE5B5BFE6400FEA9
:101E2000FE0253AD5B135252FE020E525CADADADDD
:101E3000FE000E0D130A540C01FE0112130E1703BF
:101E4000FEFEFEFE120101FEFEFEFEFE090AFEFE81
:101E5000FEFEFEFE120AFEFEFEFE00FE120AFE005E
:101E6000FEFEADA45B5CA4AD010254A45BADAD5419
:101E700002010E0E0B0B0E0E01FE020413120402E1
:101E8000FEFEFEFE0900FEFEFEFE010D03FEFEFE4E
:101E9000FEFE0C0E0000FEFEFE090B0CADADADFE0D
:101EA000FE00125C5B5B5B1309120B0CADADAD0069
:101EB00000FE030E005200FEFEFE010D03FEFEFEBC
:101EC000FEFEFEFE0200FEFEFEFE010D0300FEFE13
:101ED000FEFE0C0E5BAD5BFEFE090B5EAD5B00FE15
:101EE000FE0012135C13131309120B5EAD5B0000AE
:101EF00000FE030EA4ADADFEFEFE010D030000FECC
:101F0000FEFEFE000200FEFEFEFE010D035200FE7C
:101F1000FEFE040EA4AD00FEFE090B0C5B52FEFE9D
:101F2000FE00125C5C13131309120B0CAD5200007F
:101F300000FE030EADAD52FEFEFE010D035B52FE30
:101F4000FEFEFE000200FEFEFEFE010D035B00FE33
:101F5000FEFE0C0EA4AD00FEFE090B0C5B5B000048
:101F6000000012135B5C131309120B0CAD5B000035
:101F700000FE030EA5AD00FEFEFE010D03A400FE53
:101F8000FEFEFE000201FEFEFEFEFEFEFEFEFEFE68
:101F9000FEFEFEFE04FEFEFEFEFEFE06050402FE42
:101FA000FEFE04170B050B04FEFE030D060501FEE5
:101FB000FEFEFE040F04FEFEFEFEFEFEFEFEFEFE24
:101FC000FEFEFEFEFEFEFEFEFEFEFEFEFEFEFEFE31
:101FD000FEFEFEFE02FEFEFEFEFEFEFE02FEFEFE19
:101FE000FEFE040A000202FEFEFE02FE0202FEFEE9
:101FF000FEFEFEFE020202FEFEFEFEFEFEFEFEFEF5
:10200000FEFEFEFEFEFEFEFEFEFEFEFE1313FEFEC6
:10201000FEFE00006E1CFEFEFE00A4A4771C52A46F
:10202000FE00F5F5655B5252FEFEFE001C090052F3
:10203000FEFEFEFE1C00FEFEFEFEFEFE1CFEFEFE82
:10204000FEFEFEFE09FEFEFEFEFEFE120AFEFEFE85
:10205000FEFEFE1C7752A452FEFEFE523FA4A4A434
:10206000FE52A452656552FEFEFE52A40026FEFEFC
:10207000FEFE52FEFE1C09FEFEFEFEFEFEFE1CFEE5
:10208000FEFEFEFEFEFEFEFEFEFEFEFEFE52FEFE1C
:10209000FEFE6E1C52A452FEFEFE097F65A4A4FE45
:1020A000FEFE5252775BFEFEFE00A452522609FE4F
:1020B000FEFE00A4FEFE2509FEFEFEFEFEFEFE095B
:1020C000FEFEFEFEFEFEFEFEFEFEFEFE52FEFEFEDC
:1020D000FEFEFE52A4F6FEFEFE137F5CA4A4FEFEEE
:1020E000FEFE6537770AFEFEFEFE52525213261C94
:1020F000FEFEA45252FEFEFE09FE005252FEFEFEFD
:10210000FEFEFEFEFEFEFEFEFEFEFEFEFEFEFEFEEF
:10211000FEFEFEA4F5FEFEFEFEFE00A4F5FEFEFEA3
:10212000FE1C6E77651C1C1C09131C1C5B0900FE41
:10213000FEFEFE525200FEFEFEFEFEA45252FEFEC7
:10214000FEFEFEFEFEFEFEFEFEFEFEFEFEFEFEFEAF
:10215000FEFE00A4FEFEFEFEFEFEF5A452FEFE12F2
:1021600000FEA4A45B2525FEFE006E3F6EFEFEFE73
:10217000FE13775252A4FEFEFEFEFE00525252FEA5
:10218000FEFEFEFE52FEFEFEFEFEFEFEFEFEFEFE1B
:10219000FEFEFEFEFEFEFE09FEFE5252FEFE2EFE7C
:1021A000FE52A4A4522FFEFEFEFEA4647700FEFEA3
:1021B000FEFE133F5B52A4FEFEFE7712525200FE5B
:1021C000FEFEFEFEFE52FEFEFEFEFEFEFEFE00FED9
:1021D000FEFEFEFEFE13FEFEFEFEFEFEFE26FEFEE2
:1021E000FEFEF5A4091CFEFEFE52A4A47752520086
:1021F000FEFE525C37525252FEFEFE776E52A4FE35
:10220000FEFEFE65FEFEFEFEFEFEFEFE09FEFEFE7C
:10221000FEFEFEFE1CFEFEFEFEFEFEFE1C00FEFEA0
:10222000FEFEFEFE1C090052FEFEF5F5655B5252F5
:10223000FEFEA4A4771C52A4FEFEFE006E1CFEFE51
:10224000FEFEFEFE1313FEFEFEFEAD5252FEFEFE2D
:10225000FEFEF6ADADFEFEFEFEFEA4ADADFEFEFE44
:10226000FE656E77B71C1C1C096565655B0009FE81
:10227000FEFE5252F6FEFEFEFEFEA452F6FEFEFEEC
:10228000FEFEA400A4FEFEFEFEFEFE0000FEFEFE1C
:10229000FEFE52A4F6FEFEFEFEFE52A4F6FEFEFE7A
:1022A000FE6E777F6E1C1C1C091C6E6E5B0909FE9E
:1022B000FEFE0052A400FEFEFEFE00A4A400FEFEF0
:1022C000FEFEFEFEFEFEFEFEFEFEFEFEFEFEFEFE2E
:1022D000FEFEFE520000FEFEFEFEFEA4F500FEFE27
:1022E000FE6E777F6E252525091C6E6E5B0909FE43
:1022F000FEFEFE525252FEFEFEFEFE00FE00FEFEFE
:10230000FEFEFEFEFEFEFEFEFEFEFEFEFEFEFEFEED
:10231000FEFEFEFEFEFEFEFEFEFEFE005200FEFE85
:10232000FE6E777F6E25252509656E6E5B0909FEB9
:10233000FEFEFE000000FEFEFEFEFEFEFEFEFEFEB7
:10234000FEFEFEFEFEFEFEFEFEFEFEFEFEFEFEFEAD
:10235000FEFEFEFEFEFEFEFEFEFEFEFEFEFEFEFE9D
:10236000FEFEFEFEFEFEFEFEFEFEFEFEFEFEFEFE8D
:10237000FEFEFEFEFEFEFEFEFEFEFEFEFEFEFEFE7D
:10238000FEFEFEFEFEFEFEFEFEFEFEFEFEFEFEFE6D
:10239000FEFEFEFEFEFEFEFEFEFEFEFEFEFEFEFE5D
:1023A000FEFEFEFEFEFEFEFEFEFEFEFEFEFEFEFE4D
:1023B000FEFEFEFEFEFEFEFEFEFEFEFEFEFEFEFE3D
:1023C000FEFEFEFEFEFEFEFEFEFEFE091C09FEFEF9
:1023D000FE00525B775B00FEFE00F6AD6E5BA4FE76
:1023E000FEFE525B655252FEFEFEFE0913FEFEFE2D
:1023F000FEFEFE0913FEFEFEFEFEFEFE00FEFEFEDB
:10240000FEFEFEFEFEFEFEFEFEFEFE1309FEFEFECC
:10241000FEFE00776EA452FEFE00526577A4A4FE75
:10242000FE00A352655BFEFEFEFE52001313FEFE8D
:10243000FEFEFEFEFE13FEFEFEFEFEFEFE00FEFEA5
:10244000FEFEFEFEFEFEFEFEFEFEFEFE5252FEFE04
:10245000FEFE6E65A4A400FEFEFE5C77B6A3FEFE43
:10246000FE00525B6E0AFEFEFE005252091C0AFE7E
:10247000FEFE0000FE0009FEFEFEFEFEFEFEFEFE6B
:10248000FEFEFEFEFEFEFEFEFEFEFE0052FEFEFE16
:10249000FE000952F552FEFEFE137F6EAD00FEFEF9
:1024A000FEFE646E651313FEFEFE5252520A0A00CF
:1024B000FEFE525200FEFEFEFEFEFEFEFEFEFEFE92
:1024C000FEFEFEFEFEFEFEFEFEFEFE00FEFEFEFE2A
:1024D000FEFE52F652FEFEFEFE095BAD5B0909FEF2
:1024E000FE1C776E65131300FE095B5B52FEFEFE59
:1024F000FEFE00A452FEFEFEFEFEFEFEFEFEFEFE00
:10250000FEFEFEFEFEFEFEFEFEFEFEFEFEFEFEFEEB
:10251000FEFE5252FEFEFEFEFEFEF5A45B0A130016
:10252000FE006E77651309FEFE1377655B00FEFE05
:10253000FE000952A352FEFEFEFEFE0000FEFEFE5D
:10254000FEFEFEFEFEFEFEFEFEFEFEFEFEFEFEFEAB
:10255000FEFE00FEFE0909FEFE52A4520A1C00FE09
:10256000FE52A4B61C09FEFEFEFE65775B5200FE1D
:10257000FEFE7765525200FEFEFEFEFE0000FEFEED
:10258000FEFEFEFEFEFEFEFEFEFEFEFEFEFEFEFE6B
:10259000FEFEFEFE120AFEFEFEFE5200130AFEFEC4
:1025A000FE52F6AD1C5200FEFE52A46E6E5252FE5A
:1025B000FEFE097764A452FEFEFE001CFEFEFEFE37
:1025C000FEFEFEFEFEFEFEFEFEFEFEFE00FEFEFE29
:1025D000FEFEFE0913FEFEFEFEFEFE0913FEFEFEDB
:1025E000FEFE525B655252FEFE00F6AD6E5BA4FE2F
:1025F000FEFE525B775B00FEFEFEFE091C09FEFE3E
:10260000FEFEFEFEFEFEFEFEFEFEA45252FEFEFE9C
:10261000FEFEADAD52FEFEFEFE09ADAD5B0909FE4C
:10262000FE656E6E5C131200FE095B5B52FEFEFEE1
:10263000FEFEA4A452FEFEFEFEFE525252FEFEFE1E
:10264000FEFEFEFEFEFEFEFEFEFEFE00FEFEFEFEA8
:10265000FEFE52A452FEFEFEFE095BAD5B0909FEC2
:10266000FE6E776E13131300FE095B5B52FEFEFED7
:10267000FEFE52A452FEFEFEFEFEFEFEFEFEFEFE2C
:10268000FEFEFEFEFEFEFEFEFEFEFEFEFEFEFEFE6A
:10269000FEFEFE5200FEFEFEFE095BB65B0909FE71
:1026A000FE6E777765131300FE09095B5200FEFE8C
:1026B000FEFEFE0000FEFEFEFEFEFEFEFEFEFEFE36
:1026C000FEFEFEFEFEFEFEFEFEFEFEFEFEFEFEFE2A
:1026D000FEFEFEFEFEFEFEFEFE09125B090909FE7D
:1026E000FE6E776E1C131200FE0909090000FEFE43
:1026F000FEFEFEFEFEFEFEFEFEFEFEFEFEFEFEFEFA
:10270000FEFEFEFEFEFEFEFEFEFEFEFEFEFEFEFEE9
:10271000FEFEFEFEFEFEFEFEFEFEFEFEFEFEFEFED9
:10272000FEFEFEFEFEFEFEFEFEFEFEFEFEFEFEFEC9
:10273000FEFEFEFEFEFEFEFEFEFEFEFEFEFEFEFEB9
:10274000FEFEFEFEFEFEFEFEFEFEFEFEFEFEFEFEA9
:10275000FEFEFEFEFEFEFEFEFEFEFEFEFEFEFEFE99
:10276000FEFEFEFEFEFEFEFEFEFEFEFEFEFEFEFE89
:10277000FEFEFEFEFEFEFEFEFEFEFEFEFEFEFEFE79
:10278000FEFEFEFEFEFEFEFEFEFEFE015401FEFE0D
:10279000FEFEFE50F950FEFEFEFEFE52A500FEFEBD
:1027A000FEFEFE00AD00FEFEFEFE5BAD5CADADFECE
:1027B000FEFEAD5C54A45BFEFEFEFEFEFEFEFEFED3
:1027C000FEFEFEFEFEFEFEFEFEFEFEFE000301FE1F
:1027D000FEFEFEFEAAFA00FEFEFEFE00A452FEFE73
:1027E000FE005B5BA400FEFEFE52ADA6AE52FEFEF6
:1027F000FE000053A5FF00FEFEFEFE000000FEFEF0
:10280000FEFEFEFEFEFEFEFEFEFEFEFEFE0001FEE3
:10281000FEFEFEFE00A95BFEFE5252005BAB50FEC8
:10282000FE5BADA5A452FEFEFE00535D5BFEFEFE08
:10283000FEFE0053AD52FEFEFEFEFE0052FEFEFE08
:10284000FEFEFEFEFEFEFEFEFEFEFEFEFEFEFEFEA8
:10285000FE0052FEFE005001FE52FF5B5BACFA022E
:10286000FEFE54A5A45250FEFEFE53AE52FEFEFEE6
:10287000FEFE00AD52FEFEFEFEFEFE00FEFEFEFE71
:10288000FEFEFEFEFEFEFEFEFEFEFEFEFEFEFEFE68
:10289000FEAD5BFEFEFEFEFEFE5CAD00525001FE94
:1028A000FE545CADA5F954FEFEA4AD00005001FE3F
:1028B000005BADFEFEFEFEFE00FEFEFEFEFEFEFE28
:1028C000FEFEFEFEFEFEFEFEFEFE5200FEFEFEFED2
:1028D000FE00AD5BFEFEFEFEFE53A65B00FEFEFEAE
:1028E000FEA5AEA4A4AA00FE52FF520052FA03FEB7
:1028F000000000FE000001FEFEFEFEFEFEFEFEFEEB
:10290000FEFEFEFEFEFEFEFEFEFEFE5B52FEFEFE36
:10291000FEFE53AD52FEFEFEFE535DA500FEFEFE22
:1029200000AD5BA45B00FEFEFE520052ABA900FEB0
:10293000FEFEFE00505B01FEFEFEFEFE000000FEFD
:10294000FEFEFEFEFEFEFEFEFEFEFEFE5200FEFE51
:10295000FE005354FF52FEFEFEADAEA55BFEFEFE32
:10296000FE5252A45BFEFEFEFEFEFE52AC00FEFED8
:10297000FEFEFE50FA50FEFEFEFEFEFE0201FEFED0
:10298000FEFEFEFEFEFEFEFEFEFEFEFEFEFEFEFE67
:10299000FE5BA4545CADFEFEFEADAD5CAD5BFEFE29
:1029A000FEFE00AD00FEFEFEFEFE00A552FEFEFE97
:1029B000FEFE50F950FEFEFEFEFE015401FEFEFE3C
:1029C000FEFEFEFEFEFEFEFEFEFEFEFEFEFEFEFE27
:1029D000FEFE00AD00FEFEFEFEFE00AE5B005150AE
:1029E00000FE015DADADABFB02FE00FF5200515198
:1029F00000FE00AD00FEFEFEFEFEFEFEFEFEFEFE42
:102A0000FEFEFEFEFEFEFEFEFEFEFEFEFEFEFEFEE6
:102A1000FEFE005B00FEFEFEFEFE01A752005151CD
:102A200000FE00ADADADABFB02FE00FF5B00005150
:102A300000FE005300FEFEFEFEFEFEFEFEFEFEFE5B
:102A4000FEFEFEFEFEFEFEFEFE0000000000000098
:102A50000000005300000000000000FF5B00515127
:102A6000000000ADADADABAA020001AF5200000006
:102A70000000005200000000000000000000000004
:102A8000000000000000000000FEFEFEFEFEFEFE54
:102A9000FEFEFEFEFEFEFEFEFEFEFEFEFEFEFEFF55
:102AA000FEFEFEFEFEFFFFFF52FEFEFEFEFEFEFFEE
:102AB000FEFEFEFEFEFEFEFEFEFEFEFEFEFEFEFE36
:102AC000FEFEFEFEFEFEFEFEFEFEFEFEFEFEFEFE26
:102AD000FEFEFEFEFEFEFEFEFEFEFEFEFEFEFEFE16
:102AE000FEFEFEFEFEFEFEFEFEFEFEFEFEFEFEFE06
:102AF000FEFEFEFEFEFEFEFEFEFEFEFEFEFEFEFEF6
:102B0000FEFEFEFEFEFEFEFEFEFEFEFEFEFEFEFEE5
:102B1000FEFEFEFEFEFEFEFEFEFEFEFEFEFEFEFED5
:102B2000FEFEFEFEFEFEFEFEFEFEFEFEFEFEFEFEC5
:102B3000FEFEFEFEFEFEFEFEFEFEFEFEFEFEFEFEB5
:102B4000FEFEFEFEFEFEFEFEFE0011241FBECFEFC7
:102B5000D0E1DEBFCDBF11E0A0E0B1E0E2EEFFE5E5
:102B600002C005900D92A638B107D9F710E1A0EA8E
:102B7000B1E001C01D92A539B107E1F714BE88E1AB
:102B80000FB6F89480936000109260000FBE0E9410
:102B9000521A811102C00E94EA19F894E3EEFCE097
:102BA00080E881932EE0EF3EF207D9F783EE9CE0B8
:102BB0009093F00E8093EF0E1092F10E81E08093CF
:102BC000080F8093090F8093070F1092F40E109254
:102BD000FA0E1092000F1092060F1092B80C10927D
:102BE000BA0C92E19093B90C90EE9093C00C94E1E2
:102BF0009093BF0C1092C40C1092C30C1092C80C8E
:102C00001092C70C8093F30E0E94C72180E790E0DA
:102C1000FC0125913491F901FF273083029620E0D1
:102C20008E399207A9F778940E94C6210E94002F3E
:102C30000C94EF2F0C9400000BE90A95F1F700912A
:102C40000D0FE6E5FCE023E0029FE00DF11DC0EA78
:102C5000D1E02091850F3CE3321B300F201751F05B
:102C600000000000A191B1911C9111930C93039568
:102C70000217C0F313E01A95F1F700C03A95D1F7A7
:102C80002090B60C3090B70C0091B20C1091B30CA0
:102C9000680138018CE1C0EAD1E04E010024309196
:102CA000B50C303009F0C6E009F0D5E009F0832F0B
:102CB00009F0610100EEA02E662778E00CD336E221
:102CC0003A95F1F700000E9494163FE03A95F1F72B
:102CD00000000000AA94A9F06395C895683031F00F
:102CE00033E03A95F1F700000000E8CF66270024B2
:102CF0003EE1C30FD01D8A9509F4E40109F4630194
:102D0000DDCF36E03A95F1F7E6D211240E942D206E
:102D1000E091BA0C42E0E160E427E093BA0CE2E013
:102D2000E093360011240895DE01679F860100506C
:102D30001740000D111D180106E515E0000D111DCD
:102D4000280130E41EE12D91239FA1012C3108F4CC
:102D5000A201040E151EF0012C31F0F0059108B906
:102D60002D91059108B9239F059108B92C310000D8
:102D7000059108B908F4A201059108B9040E151EC1
:102D8000059108B92C311A95059108B9059131F1D1
:102D9000F00108B918F700C0019108B92D9101910F
:102DA000000008B9239F0191000008B92C3100C030
:102DB000019108B908F0A1010191040E08B9151E8E
:102DC00000C0019108B92C3100C0019108B90191EE
:102DD0001A9521F0F00108B908F6DECF08B90027EE
:102DE000C895000008B9089520E4E091B20CF09174
:102DF000B30C829FE00DF11DA6E5B5E0629FA00D2A
:102E0000B11D15901D9215901D9215901D92159053
:102E10001D9215901D9215901D9215901D92159062
:102E20001D9215901D9215901D9215901D92159052
:102E30001D9215901D9215901D9215901D92159042
:102E40001D9215901D9215901D9215901D92159032
:102E50001D9215901D9215901D9215901D92159022
:102E60001D9215901D9215901D9215901D92159012
:102E70001D9215901D9215901D9215901D92159002
:102E80001D9215901D9215901D9215901D921590F2
:102E90001D9215901D9215901D9215901D921590E2
:102EA0001D9215901D9215901D9215901D921590D2
:102EB0001D9215901D9215901D9215901D921590C2
:102EC0001D9215901D9215901D9215901D921590B2
:102ED0001D9215901D9215901D9215901D921590A2
:102EE0001D9215901D9215901D9215901D92159092
:102EF0001D9215901D9215901D9215901D92159082
:102F00001D921124089520E4E6E5F5E0829FE00D8E
:102F1000F11DA6E5B5E0629FA00DB11D11901D92B7
:102F200011901D9211901D9211901D9211901D9261
:102F300011901D9211901D9211901D9211901D9251
:102F400011901D9211901D9211901D9211901D9241
:102F500011901D9211901D9211901D9211901D9231
:102F600011901D9211901D9211901D9211901D9221
:102F700011901D9211901D9211901D9211901D9211
:102F800011901D9211901D9211901D9211901D9201
:102F900011901D9211901D9211901D9211901D92F1
:102FA00011901D9211901D9211901D9211901D92E1
:102FB00011901D9211901D9211901D9211901D92D1
:102FC00011901D9211901D9211901D9211901D92C1
:102FD00011901D9211901D9211901D9211901D92B1
:102FE00011901D9211901D9211901D9211901D92A1
:102FF00011901D9211901D9211901D9211901D9291
:1030000011901D9211901D9211901D9211901D9280
:1030100011901D9211901D9211901D9211240895EE
:103020000F931F93CF93DF9394E0899FE6E0F5E041
:10303000E00DF11D03818281E0E48E9FD00198E0D4
:10304000099FCAEADCE00024C10DD01DE881F981A6
:10305000EA0FFB1FA6E5B5E090E4699FA00DB11D46
:103060001124DD27403051F4A20FB11D822FC22F51
:1030700000FF11C03796C0E1C21B0DC088E0821B63
:1030800000FD04C0C82FE80FF11D05C0C8E0C20F45
:10309000E20FF11D3197503051F498E0939FA00D4D
:1030A000B11D932F01FDE85C01FDFF4F0AC098E0C0
:1030B000931B632F6A9501FF692F58E0569FE00D1F
:1030C000F11D6FEF7FEF00FF61E000FF772701FD4B
:1030D000609711243EEF58E0591B48E0481B2491AB
:1030E00023132C931196E60FF71F4A95C1F7EC0FA7
:1030F000FD1FA80FB11D5A9581F7DF91CF911F9148
:103100000F9108950F921F92EF93FF93EFB7EF93F4
:10311000E0918400E251F1E0EF1700F0F395FA300E
:10312000D8F30C949318E091B90CEA95E093B90C9C
:10313000F091B80CF0FD57C0EC3098F0F3E0F0934C
:103140008900FDE8F0938800E0FB289826F4E1E090
:103150000E940220B9C0E5E1EA95F1F70000289A43
:10316000B3C0E63038F100C000C02898E0FBE4E0CE
:1031700016F40E940220E4E0E0933600E6E0E093DB
:103180006F00A2C0EF93EFB7EF93E0918400ED558D
:10319000E13000F0E23000F0E33000F0E43000F025
:1031A000E53000F0289AE2E0E0936F00EF91EFBF86
:1031B000EF91189500C0E0FB289826F4E1E00E940A
:1031C000022005C0E5E1EA95F1F70000289AE091B8
:1031D000B90CE03009F078C0EDEFE093B90CE1E014
:1031E000E093B80C71C0E7E0E0938900EBE1E09375
:1031F000880000C02898E2E000C00E940220FDEF95
:103200000090BF0CF019E091B90CEF17E0F4FDEF5E
:103210000090BF0CF0190090C00CF019EF1798F057
:10322000EDE1FF2700800F92EA95E1F70FE10A95A3
:10323000F1F7000000000E941C16E1E0FF270F904C
:103240000192EE31E0F3E091B90CE03009F03CC0BE
:103250002F933F934F935F936F937F938F939F939E
:10326000AF93BF9378941124EE27E093B80CE2E17A
:10327000E093B90C8091C90C9091CA0C019680938F
:10328000C90C9093CA0CE091BB0CF091BC0CE115F9
:10329000F10509F009950E94BD190E940F240E94B2
:1032A0004A1F1124E091BD0CF091BE0CE115F1050F
:1032B00009F00995BF91AF919F918F917F916F9187
:1032C0005F914F913F912F91EF91EFBFFF91EF9160
:1032D0001F900F9018952898E2E000C00E940220ED
:1032E000E091B90CEA95E093B90C089528E088E1E3
:1032F00090E00FB6F894A895809360000FBE2093DD
:103300006000FFCF6093C00C8093BF0C0895129AA9
:10331000C895C895C895C895129840E180E090E09E
:1033200020E030E03695279596958795C895C89505
:10333000C895C8951398009B3068019B9068139AB4
:10334000C895C895C895C895415061F73093C20C8F
:103350002093C10C9093C60C8093C50C8091C10C36
:103360009091C20C0F9731F08091C50C9091C60CD2
:103370000F9711F40E94761908951092160F009974
:1033800003C081E08093160F019905C08091160F4C
:1033900082608093160F0E94871908952091160F5E
:1033A00020FF0BC08091C10C9091C20C9095991F89
:1033B0009927991F82E0891B01C080E021FF09C085
:1033C0002091C50C3091C60C37FF02C0886008956B
:1033D00084600895CF93DF93C0E0D0E0FE01E25611
:1033E000FF4F6491CE010E94262B2196C032D10559
:1033F000A9F7C0E2D0E06FEFCE010E94262B6FEF5D
:10340000CE0101960E94262BA096C11588E0D80710
:1034100091F7DF91CF910895A0E0B0E0E2E1FAE109
:103420000C94C22FE82ED92EF62EC0E0D0E0FE017B
:10343000E256FF4F6491CE010E94262B2196C830A0
:10344000D105A9F7C0E2D0E0CE010E94302BC82EF2
:103450008E010F5F1F4FC8010E94302B282F30E0D4
:10346000322F22272C0D311DEE2DFD2D80E08F15E2
:1034700039F0419151912417350751F08F5FF7CF03
:103480006FEFCE010E94262B6FEFC8010E94262B02
:10349000A096C11588E0D807B9F6CDB7DEB7E8E049
:1034A0000C94DE2FCF9380E090E00E94302BC82F49
:1034B00081E090E00E94302B282F30E0322F22272D
:1034C0002C0F311D81E02A35354509F080E0CF9180
:1034D000089599B19C7081E09C3009F480E00895D2
:1034E000A0E0B0E0E6E7FAE10C94BE2F8C017B018E
:1034F0006A01FB01118210828F3FFFEF9F0771F17C
:10350000C0E0D0E0B12CA3E09A2EA12CCE010E9405
:10351000302B882ECE0101960E94302B282F30E0D0
:10352000322F2227280D311D2017310729F4F701EA
:10353000D183C083912C0BC02F3F3F4F41F4A1108A
:1035400006C0C114D10411F0F601B082AB2CB394C3
:10355000A096F0E4BF12DACF892D01C081E0CDB78B
:10356000DEB7ECE00C94DA2FA3E0B0E0EAEBFAE18E
:103570000C94C42F8C011A8219821B82AE014D5FFC
:103580005F4FBE016F5F7F4FFC01808191810E9480
:10359000701A882311F0833021F589819A81892B53
:1035A00049F48B818823D1F0F0E28F9FC001112470
:1035B0009A838983780120E2E20EF11CF80161917F
:1035C0008F0189819A819C012F5F3F4F3A83298324
:1035D0000E94262B0E151F0589F702C082E001C04C
:1035E00080E02396E6E00C94E02FA2E0B0E0EBEF61
:1035F000FAE10C94C32F8B0140E050E0BE016F5FF5
:103600007F4F0E94701AD82E811113C0780180E27A
:10361000E80EF11C89819A81AC014F5F5F4F5A839C
:1036200049830E94302BF80181938F01EE15FF052D
:1036300089F78D2D2296E7E00C94DF2F009721F07B
:103640009093E10C8093E00C2091E00C3091E10C20
:10365000C9019695879596958795A90163E056953A
:1036600047956A95E1F78427952782279327A90133
:1036700075E0569547957A95E1F784279527992720
:1036800086959795882736952795822B932B90932F
:10369000E10C8093E00C0895FC016787089581E0B8
:1036A00091E09093090F8093080F6093070F08959E
:1036B000FC0120812F7520830895FC012081206466
:1036C00020830895FC0166870895FC0162870895B0
:1036D000FC0163870895CF93DF93EC01462F298186
:1036E00030E0C901880F991F885F984AFC016591F5
:1036F0007491F901E40FF11D47FDFA95EE0FFF1FDC
:10370000E85FF84A85919491861B970B688570E075
:103710000E94822F6115710511F461E070E0EA8169
:1037200086E0E89FF0011124EC50F14F21813281B5
:10373000260F371F328321837E836D8388818860C3
:1037400088838981840F8F83DF91CF910895FC0155
:1037500060870895FC0164830895FC0182810E94C2
:10376000502B0895FC018181680F618382810E9442
:10377000392B0895FC018181861B8183682F82810A
:103780000E94392B08951F93CF93DF93EC01162FDE
:103790008A810E94392B19838881877F8883DF91F2
:1037A000CF911F910895DC0114962C911497222338
:1037B00039F15596ED91FC9156976623A1F0772744
:1037C00067FD70956F5F7F4FCB01880F991F860F44
:1037D000971FE81BF90B5696FC93EE9355970DC077
:1037E000EF3F39F0FC01CF0103973597E491ED30BD
:1037F000B9F756969C938E935597215014962C9317
:1038000008959093780F8093770F8FE680937A0FC7
:103810001092E20CE9E2FFE080E090E13FEF28E166
:10382000DF011E978C93DF0150979C93DF01139764
:103830001C92DF0114973C931082DF0115972C93A3
:10384000DF0118979C938F5F7796843049F708952E
:10385000E9E1FFE0ACE1BFE03FEF20812F7720837B
:103860003C93779657962FE0E537F207B1F701962C
:1038700090937F0F80937E0F9093180F8093170F74
:103880009093810F8093800F10927C0F10927B0F8A
:103890001092760F1092750F10927D0F1092790F83
:1038A00081E08093E20C08958AEF8093280F809343
:1038B0003F0F8093560F80936D0F1092E20C089586
:1038C00081E08093E20C089580937D0F08958091AC
:1038D0007D0F0895DC01ED91FC9111979F012F5F01
:1038E0003F4F11963C932E93849187FD02C090E048
:1038F00008958F7790E0F9019695982F88279795EE
:1039000087952F5F3F4FE4914E2F4F77840F911D86
:10391000E7FDF1CF2D933C9308950F931F93CF9321
:10392000DF93EC01162F9881092F001F0027001F3D
:103930001F868FEF8E874D871C8A977B98831A8608
:10394000198629831C828B838A81833069F4011153
:1039500001C0122F81E091E09093090F8093080F2E
:1039600081E08093070F07C0622F0E94392B60E02F
:103970008A810E94502B002311F0198B01C0188BF3
:10398000E091770FF091780F89E0189FE00DF11D1D
:103990001124339685919491009719F41E8A1D8AFB
:1039A00007C01B8AFC0124912A8B01969E8B8D8B6C
:1039B000DF91CF911F910F910895CF93DF93E09105
:1039C000770FF091780F99E0899FE00DF11D112498
:1039D000E491E130F9F0E230F9F02091300F27FD69
:1039E00002C0C1E01CC02091410F281302C0411148
:1039F000F8CF2091470F27FF11C02091580F2813AF
:103A000002C041110BC02091440F90915B0F92179F
:103A100028F4E7CFC3E003C0C4E001C0C2E097E1EF
:103A2000C99FE0011124C75ED04F90E898831E8A99
:103A30001D8A20E5462F682FCE010E948D1C8881AB
:103A400080628883DF91CF910895CF93DF93922F87
:103A500027E1829FE0011124C75ED04F888185FF56
:103A600002C087FD14C0911107C09F85911102C04B
:103A700086FF1D868F7B0AC018821E8A1D8A242F0E
:103A8000492FCE010E948D1C888180628883DF913E
:103A9000CF910895A0E0B0E0E0E5FDE10C94C02FE7
:103AA000A5EFBEE0C9E1DFE020E030E0F901E75E2C
:103AB000F04F8785882389F04685992787FD909563
:103AC000840F911D8F3F910519F014F08FEF90E056
:103AD00097FF02C080E090E08687188113FF23C023
:103AE0006D817E818D919C911197860F971F119604
:103AF0009C938E93E781F0E0EE0FFF1FE85FF84A9A
:103B0000459154911616170624F48417950730F43E
:103B10000AC0672B41F04817590728F011965C93AB
:103B20004E93177F1883295E3F4F679616962C3564
:103B3000310509F0BBCF8091E20C882309F4C6C09F
:103B4000C7E18091750F9091760F20917B0F309196
:103B50007C0F8217930709F0B4C020917E0F30913B
:103B60007F0FB9016F5F7F4F70937F0F60937E0F60
:103B7000F90144914F3F69F5A9014E5F5F4F5093A2
:103B80007F0F40937E0FFB0164916F3219F4109206
:103B9000E20C97C0663009F087C0C9010496909383
:103BA0007F0F80937E0FF90133962491233529F4FA
:103BB0009093810F8093800F77C0253409F074C0F3
:103BC0008091800F9091810F90937F0F80937E0F53
:103BD0006BC047FD4093790F9091790F892F8F70BB
:103BE00047FF08C02E5F3F4F30937F0F20937E0F1B
:103BF000FB014491907F903BE9F0903C09F44EC06A
:103C0000903909F051C0E0917E0FF0917F0F9F0134
:103C10002F5F3F4F30937F0F20937E0F2491220F11
:103C2000C89FD0011124A75EB04F50966C910E949E
:103C3000251D3AC0E0917E0FF0917F0F9F012F5F0D
:103C40003F4F30937F0F20937E0F9491473041F484
:103C5000C89FF0011124E75EF04F990F948724C0AC
:103C60004B3041F4C89FF0011124E75EF04F990FEB
:103C700093831AC04C3541F4C89FF0011124E75ECC
:103C8000F04F990F928710C0443671F4C89FF0012D
:103C90001124E75EF04F990F938706C0C89FF0018B
:103CA0001124E75EF04F408B8EE79FE00E946A1C74
:103CB00090937C0F80937B0F1092760F1092750F6C
:103CC00040CF01969093760F8093750F44EFA42E0A
:103CD0004EE0B42EC9E1DFE000E010E0CC24CA944D
:103CE000D12C288125FF43C08D899E89892B09F419
:103CF0003EC026FD3CC0C801875E904F7C01F701A5
:103D00002389828928132FC0ED89FE89BF016F5F47
:103D10007F4F7E8B6D8B34913F3F31F488818F775D
:103D200088831E8A1D8A1FC0CF0102969E8B8D8BB1
:103D3000FB016491E32FF0E0EE0FFF1FE254FF4F11
:103D400025913491CE01F9010995ED89FE89CF01C4
:103D500001969E8B8D8BE491D7015296EC935297EE
:103D600053961C92CCCF2F5FD70153962C9388810A
:103D700085FF74C0D801A75EB04F54969C915497AC
:103D80009F3F21F09F5F54969C93549787FD04C0FA
:103D90001C968C911C9701C08FEF1D962C911D973E
:103DA00019966C911997222309F44FC01E965C91C5
:103DB0001E97552309F449C0882309F446C0409151
:103DC0007A0F442309F441C0289F900111243395B0
:103DD000232F3327529FC001539F900D1124939599
:103DE000892F992713965C911397589F9001599F9B
:103DF000300D11243395232F3327429FC001439F59
:103E0000900D11249395892F99271A962C911A9722
:103E10002223E9F0E62FF0E0E050F74AE491E05881
:103E20002E9FF0011124F395EF2FFF27A6014E1BC3
:103E30005F0B489F9001499F300D589F300D112412
:103E4000C9019395892F992702C080E090E01B96C5
:103E50002C911B97260F19962C9302C080E090E0BE
:103E6000F5018083095E1F4F6796F6E0AF0EB11C27
:103E70000C35110509F035CFCDB7DEB7EAE00C946B
:103E8000DC2F80937A0F089580917A0F08958091A6
:103E9000E20C0895E091F30EE0FD0E944A1D0090AF
:103EA000F10E002019F4A3EEBCE002C0A9EEBDE0C3
:103EB00021E002260092F10E22E02093F20EE09122
:103EC000F30EE0FF08952F923F924F925F926F9210
:103ED0007F928F929F92AF92BF92CF92DF92EF929A
:103EE000FF920F931F93CF93DF932090F50E3090A6
:103EF000F60E4090F80E5090F90E6090F70E10916B
:103F0000F40E7090FB0E8090FC0E9090FD0EA09031
:103F1000FE0EB090FF0E2091FA0EC090010FD090CF
:103F2000020FE090040FF090050F0091030F309105
:103F3000000F9FEF620C431CF20144914103000803
:103F4000C12DD02D970CA81CF50144914203000807
:103F5000C10DD01D0C0DED1CF70144914303000869
:103F6000C10DD01D0024C038D0050CF0CFE70A9455
:103F7000C038D0050CF4C0E8C058CD939A9509F02C
:103F8000D9CF4091F20E4A954093F20E97E009F096
:103F9000D1CF6092F70E4092F80E9092FD0EA09253
:103FA000FE0E0093030FE092040F6093080F7093CE
:103FB000090F80930A0FDF91CF911F910F91FF900E
:103FC000EF90DF90CF90BF90AF909F908F907F90B9
:103FD0006F905F904F903F902F900895E091EF0E7B
:103FE000F091F00E019100000093B3000EE0EF3E5F
:103FF000F00703EE1CE008F0F801E093EF0EF093F9
:10400000F00E08950F931F932F93EF93E091EF0E0F
:10401000F091F00E01910093B3000EE0EF3EF00737
:1040200003EE1CE008F0F801E093EF0EF093F00EC1
:10403000E8E0EA95F1F7EF912F911F910F91E0FDE4
:10404000289AE0FF01C00895F4E1FA95F1F700C065
:10405000E1FD289AE1FF00C0089520910D0F8091A5
:10406000850F281778F4822F90E0FC01EE0FFF1FD8
:10407000E80FF91FEA5AF34FA081B18182818C9336
:104080002F5FEDCF089580930C0F089520E4829F59
:10409000C00111248A5A9A4F08958093000108950F
:1040A000A6E0B0E0E6E5F0E20C94B82F80910001C4
:1040B000882309F4B1C080910C0F80930D0F809379
:1040C000850FE7E0EE2EE5E0FE2E512CF70131974B
:1040D0002081203F09F497C0F7013081832F90E0C1
:1040E000222E269426942694277019F4F1E0F98361
:1040F00002C042E0498373E0969587957A95E1F78F
:10410000382E832F877011F491E001C092E09A83DA
:10411000C82ED12CDC2CCC24C20ED11C00E010E027
:1041200093EE930D9B8392EE920D9C83832D800FD3
:104130008D3118F08B80800E01C0882EEEE18E9EAE
:1041400040011124B02EAA241E821D828D81820D71
:104150008E3118F08C81ED818E0F3401680E711C48
:10416000C30180569E4F3C01FC01408081E0FBE191
:10417000F41508F080E091E020910D0F421618F040
:1041800090E0882341F16091850F6C3108F5882318
:1041900029F084EE840D0E94F41605C0992319F0CD
:1041A000842D0E9483178091850F282F30E0F9011C
:1041B000EE0FFF1FE20FF31FEA5AF34F7182608286
:1041C0004282F301808391E0980F9093850F482EEF
:1041D000FBE1F41548F096014D815E814A0D5B1DAF
:1041E000642D852D0E9410188D819E8101969E83DD
:1041F0008D839981891708F4A9CF0F5F1F4F9A818A
:10420000091708F493CF5394F4E0EF0EF11C44E146
:1042100054125CCF0E942D202696E2E10C94D42FFC
:10422000FF920F931F93CF93DF93FB01149131966D
:104230000491412F50E090E0861BF82EF60E901767
:10424000D9F020E030E0EB012296AF2DA20F21172C
:1042500078F4FE01E20FF31FE491F4E0AF9FD00188
:104260001124AA5FBA4F1296EC932F5F3F4FEDCF08
:104270009F5F640F751FE1CFCDB7DEB7E5E00C940B
:10428000E12FA0E0B0E0E7E4F1E20C94C12FFB01E4
:1042900014913196D490CC24CA94C10E242F21704D
:1042A00040FF04C09C2DFF24FA9403C0FF24F39424
:1042B00090E041FF05C05FEF5D0DEE24EA9403C07E
:1042C000EE24E39450E0211101C0C12C00E00D1553
:1042D00011F15103E0011124B82EB10E8B15B9F084
:1042E000FE01E90FF11D97FDFA953296E60FF71FD3
:1042F0002491F4E08F9FD0011124AA5FBA4F129647
:104300002C9312978F5F13964C939F0DE7CF5E0D02
:104310000F5F9C2DDCCFCDB7DEB7E9E00C94DD2F2D
:10432000A0E0B0E0E6E9F1E20C94C22FE0E0F0E0BA
:1043300030E0A8E1DA2ED40EE42EF12C301709F18A
:104340001D2D1E0F742F7E0FC82EC20E962FEF014B
:10435000CE0DDF1D8C1591F054E0859FD001112406
:10436000AA5FBA4F9C93C93ED1051CF011961C93CD
:1043700002C011967C938F5F985FECCF3F5F3896B9
:10438000DDCFCDB7DEB7E8E00C94DE2F0895E6E090
:10439000F5E080EF8083349695E0E635F907D1F7B4
:1043A0000895A0E0B0E0E7EDF1E20C94BC2F682E98
:1043B000862EFA01A49031967490CA2CD12C8A01D1
:1043C000B12CB714D1F0C0E0D0E0780182E0E80E63
:1043D000F11C9B2C980CCA1560F4F701EC0FFD1F23
:1043E000449150E0692D8C2F860D0E94FA2A219667
:1043F000F2CFB3940C0D1D1DE4CFCDB7DEB7EEE0C8
:104400000C94D82FA0E0B0E0E8E0F2E20C94BD2FCD
:10441000062F69017A01EC01219710E0BAE08B2E9A
:10442000912CA12CB12C7C2E7394C114D104E104E5
:10443000F10411F4111109C0C701B601A5019401DD
:104440000E94962F40E1460F01C040E0602F872D6B
:104450000E94F62AC701B601A50194010E94962F79
:1044600069017A011F5F21971A30E9F6CDB7DEB7EF
:10447000EDE00C94D92FA0E0B0E0E1E4F2E20C947E
:10448000C32FF62E042FD22EEC01219710E08AE0E4
:10449000E82E3C2F3F5F011102C0111107C0802F91
:1044A0006E2D0E94542F905F492F05C0DD2011F022
:1044B00040E101C040E06F2D832F0E94F62A802F3B
:1044C0006E2D0E94542F082F1F5F2197133009F77C
:1044D000CDB7DEB7E7E00C94DF2FA0E0B0E0E3E774
:1044E000F2E20C94C12FC62EEA01B22E8C010150CB
:1044F0001109D12C9AE0E92EF12C31E0300F2097F0
:1045000011F4D11007C0CE01B7010E946E2F40E117
:10451000480F05C0BB2011F040E101C040E06C2D08
:10452000832F0E94F62ACE01B7010E946E2FEB0165
:10453000D3940150110985E0D812DFCFCDB7DEB793
:10454000E9E00C94DD2F0F931F93CF93DF93162F89
:10455000D42FC82F08E0080FD7FF02C041E101C0E7
:1045600040E1612F8C2F0E94F62ADD0FCF5FC01330
:10457000F3CFDF91CF911F910F9108951F93CF93A8
:10458000DF93D82FC62F142F842F82958F708A30F7
:1045900010F440E101C047E1480F6C2F8D2F0E94BD
:1045A000F62A412F4F7081E08D0F4A3010F4405FA2
:1045B00001C0495E6C2F0E94F62ADF91CF911F91B6
:1045C00008951F93CF93DF93C82FD62F142F452F15
:1045D0000E94BE22412F6D2F82E08C0F0E94BE22CE
:1045E000DF91CF911F910895CF92DF92EF92FF92CA
:1045F000CF93DF93C82FD62F69017A014F2D55270E
:10460000662777276D2F0E94BE22A701662777278E
:104610006D2F82E08C0F0E94BE2277276F2D5E2DBA
:104620004D2D6D2F84E08C0F0E94BE224C2D6D2FDE
:1046300086E08C0F0E94BE22DF91CF91FF90EF9019
:10464000DF90CF9008950F931F93CF93DF93162F92
:10465000C42FD52F082F041BFE014491442349F099
:104660004F774052612F8C2F800F0E94F62A21969F
:10467000F3CFDF91CF911F910F9108950F931F9367
:10468000CF93DF93062FC42FD52F142F1095180F1B
:104690004991442341F04F774052602F8C2F810F76
:1046A0000E94F62AF5CFDF91CF911F910F910895C7
:1046B00040520E94F62A0895A0E0B0E0E2E6F3E25C
:1046C0000C94BD2F882E962E6A015901C0E0D0E0CF
:1046D000CA15DB059CF4E12CF12C7C2E790CEC1432
:1046E000FD0454F4A801672D882D8E0D0E94FA2A2E
:1046F0008FEFE81AF80AF3CF2196EACFCDB7DEB7ED
:10470000EDE00C94D92FA0E0B0E0E9E8F3E20C94DE
:10471000BE2F982E162F6A015901C0E0D0E000523A
:10472000CA15DB059CF4E12CF12C8C2E810EEC14C7
:10473000FD0454F4402F682D892D8E0D0E94F62A19
:104740008FEFE81AF80AF3CF2196EACFCDB7DEB79C
:10475000ECE00C94DA2F0F931F93CF93DF938C012F
:10476000C0E0D0E0C017D10744F40E94102B88238A
:10477000E1F30E94142B2196F5CFDF91CF911F9189
:104780000F9108958093830F1092870F81E080939B
:10479000860F662321F08091860F8111FCCF08954A
:1047A000811103C08FEF87B9089591E09093880F2E
:1047B0009093840F0E94C2230895811102C017B8FC
:1047C00008959CE09093880F9FEF9093840F0E9430
:1047D000C22308958091860F882301F18091870F6D
:1047E000811119C08091830F8093870FE091880F0A
:1047F000F0E0E552FF4FE491E7B98091840F90918A
:10480000880F890F8093880F882311F08D3031F441
:104810001092860F089581508093870F08950E940B
:10482000EA230E9450200895E0914D01E150E09369
:104830004D01FF27E7FDF095E25BFE4F8081089573
:10484000A1E0B0E0E6E2F4E20C94C62F95E0969F7A
:104850008001979F100D11240757104FD801139610
:104860008C93139714961C92149711964C9311974E
:1048700081E08C9349830E941424F801828394E0A0
:104880008902F0011124EA5FFA4F4981405C4283BA
:104890002196E4E00C94E22FCF93DF9380911D01E9
:1048A00090911E0188539F4F2091140F3091150F46
:1048B000821793070CF04AC080910E0F90910F0F52
:1048C00002970CF043C0EAE8FFE0C0E0D0E040818E
:1048D0008FEF840F8E3FA8F5DF0111978C91811126
:1048E00030C0BE0183E00E94202485E08C9FF0014F
:1048F0008D9FF00D1124E757F04FE28184E0E8022C
:10490000F0011124EA5FFA4FCE0166EF7FEF0E94BB
:10491000822F625F7F4F6295607F6083CE016AE085
:1049200070E00E94822F02968295807F8183809121
:104930000E0F90910F0F019690930F0F80930E0F13
:1049400005C021963596C233D10509F6DF91CF9186
:104950000895CF938091140F9091150F6091130FCC
:10496000262F332727FD309577E0729FF001739F44
:10497000F00D1124E95FFE4F4181528184179507A4
:10498000C1F4A9014F5F5F4F749FF001759FF00D57
:104990001124E95FFE4F71E0418152818417950730
:1049A00009F070E07093120F1092060144E04093FA
:1049B00005018F3245E794072CF401969093150F6B
:1049C0008093140F64300CF05BC08091060181115C
:1049D00050C085E0809306018091050118160CF007
:1049E00048C0815080930501C7E0C29FF001C39F7A
:1049F000F00D1124E95FFE4FDF01A80FB11D1396E2
:104A00006C91772767FD709541E080810E9420249A
:104A10008091120F8823E9F08091130F992787FD69
:104A20009095019620910501C89FF001C99FF00D56
:104A30001124E95FFE4FDF01A20FB11D27FDBA95DA
:104A400013966C91772767FD709541E080810E94F5
:104A500020248091050181110CC09091130F809149
:104A6000120F882311F082E001C081E0890F80934A
:104A7000130F8091060118161CF4815080930601D3
:104A8000CF91089590914D01E92FFF27E7FDF09513
:104A9000E25BFE4F80839F5F90934D01089525E078
:104AA000289FF001299FF00D1124E757F04F148241
:104AB000E28124E0E202F0011124EA5FFA4F218151
:104AC00030E0283431059CF02139310534F440912F
:104AD000070550E04217530754F425E0289FF001E2
:104AE000299FF00D1124E757F04F82E409C025E01B
:104AF000289FF001299FF00D1124E757F04F82E025
:104B0000838308958F929F92BF92CF92DF92EF920C
:104B1000FF920F931F93CF93DF931F92CDB7DEB712
:104B20009C0166EF7FEF0E94822F625F7F4FC62E4F
:104B3000CC0CC9016AE070E00E94822F0296682FB7
:104B4000660F85E0829F8001839F100D1124075717
:104B5000104FF8018281F4E08F0240011124F4012A
:104B6000EA5FFA4FB08098E0C99E900111242B199A
:104B70003109D18098E0699FA00111244D19510994
:104B8000449FD001459FB00DB00D1124229F7001AC
:104B9000239FF00CF00C1124AE0DBF1D199770F47B
:104BA00090EF908369830E94422545EA50E0698135
:104BB0008C2D0E94FA2AF8011082A9C02115310516
:104BC00021F41416150694F073C064E6649FC001C6
:104BD000659F900D1124B9010E94822F12161306B1
:104BE0000CF062C0693682E078071CF083E08D0D1E
:104BF000BFC0633A710544F083E08D0D8183B394A7
:104C0000B0828DE090E0B7C06F3371054CF0D39463
:104C1000D394D182B394B394B0828EE090E0ABC0D1
:104C20006C30710544F0D394D18283E08B0D808386
:104C30008FE090E0A0C0663F9FEF790734F083E0FB
:104C40008B0D808380E090E096C0633C8FEF780707
:104C500044F0DA94D18283E08B0D808381E090E090
:104C60008AC06F359FEF790764F0F401EA5FFA4F6D
:104C7000DA94DA94D18280818E5F808382E090E042
:104C80007AC08DEF8D0D69397D4F54F0F401EA5FE4
:104C9000FA4F818380818F5F808383E090E06BC0D7
:104CA000F401EA5FFA4F06C0693682E0780734F013
:104CB0008DEF8D0D818384E090E05DC0633A7105D6
:104CC00044F08DEF8D0D8183BA94B08285E090E041
:104CD00052C06F3371054CF0DA94DA94D182BA94F1
:104CE000BA94B08286E090E046C06C30710544F022
:104CF000DA94D1828DEF8B0D808387E090E03BC00A
:104D0000663F9FEF790734F08DEF8B0D808388E04D
:104D100090E031C0633C8FEF780744F0D394D182A8
:104D20008DEF8B0D808389E090E025C06F359FEF7C
:104D3000790764F0F401EA5FFA4FD394D394D182F7
:104D40008081825080838AE090E015C083E08D0DE1
:104D500069397D4F54F0F401EA5FFA4F8183808115
:104D6000815080838BE090E006C0F401EA5FFA4F47
:104D700081838CE090E0F401EA5FFA4F2AE9228314
:104D80008430910514F49EE909C08D3091052CF40E
:104D90008A56828381E0838304C09EEA981B9283B3
:104DA00013820F90DF91CF911F910F91FF90EF90A1
:104DB000DF90CF90BF909F908F90089587FD80588F
:104DC000282F332727FD3095803224F4F901E45A47
:104DD000FE4F06C0803434F4EBE9F1E0E21BF30B44
:104DE00080810895803624F4F901E45EFE4F04C00A
:104DF000EBEDF1E0E21BF30B808181950895A2E0D9
:104E0000B0E0E5E0F7E20C94BE2F8C0185E0809FD6
:104E1000F001819FF00D1124E757F04F84818F3FFF
:104E200011F08F5F848385E0809FF001819FF00DFA
:104E30001124E757F04FC280DD24C7FCD0942381B2
:104E4000822F8F734481322F3074932E26FD4C5F56
:104E500081116CC0403438F504E710E0041B1109DF
:104E6000000F111F80E2840F49830E94DE2690E824
:104E7000E92EF12CE81AF10887FDF3944981842F7B
:104E80000E94DE26992787FD9095BC01605F7F4FC9
:104E900077FF03C0BC01615D7F4FA5E07595679505
:104EA000AA95E1F731C0403690F5E42EF12C570178
:104EB00040E4A41AB1088A2D880F0E94DE2687FDDF
:104EC0008F5F859508E610E0081B110987FD139593
:104ED000C701C097880F0E94DE2687FD8F5F8595EA
:104EE000E82EFF24E7FCF09450EAE50EF11CB7FE33
:104EF00003C083E0A80EB11CB50175956795759543
:104F00006795719561957109685F7F4F27C140373B
:104F100008F05CC1042F10E00C521109000F111FA2
:104F200060E070E0E0E8EE2EF12C18C1813009F06D
:104F30005FC0403290F5042F10E00C5E1F4F000F51
:104F4000111F842F49830E94DE26E4E08E02C001F7
:104F5000112463E070E00E94822F7B01F9E0EF0EE4
:104F6000F11C498180E2840F0E94DE26992787FD8B
:104F700090959C01205F3F4F37FF03C09C01215D4E
:104F80003F4F45E0359527954A95E1F76627772706
:104F9000621B730B6F707727E1C0403608F016C1B3
:104FA000A42EB12CC50180549109880F0E94DE26E1
:104FB00087FD8F5F859508E610E0081B110987FDC6
:104FC0001395C501C097880F0E94DE2687FD8F5F6D
:104FD000859590E4E92EF12CE81AF10887FDF39409
:104FE000B501605271097595679575956795B6C05D
:104FF000833069F5E42EF12CC7014096880F498370
:105000000E94DE26B5E18B2E682D0E94602FA82E0F
:10501000BB24A7FCB094C7018096880F0E94DE26AF
:10502000682D0E94602FE82EFF24E7FCF094498150
:10503000642F6695669570E0403209F0CBC0C801D8
:1050400069837A830E944F2569817A81C3C0823047
:1050500009F052C0433070F04930C0F04F3098F042
:10506000453170F04B3148F0413250F0473258F042
:105070004D3260F068E070E00BC06CE070E008C09A
:105080006BE070E005C06AE070E002C069E070E0CB
:10509000CB010897FC01EF57FE4FA080BB24A7FC73
:1050A000B094FC01E458FE4FE080FF24E7FCF0944C
:1050B000403339F4C80169837A830E944F257A818D
:1050C0006981F601EE0FFF1FEE0FFF1FEA5FFA4F37
:1050D000808181117FC085E0809FD001819FB00DCC
:1050E0001124A757B04F84E013968C93139714960E
:1050F0001C9288E780836EC08430B1F49601220F41
:10510000331F220F331FF901EA5FFA4F493C18F0B1
:1051100085EA82835BC082E8828368E070E0E12CEC
:10512000F12C00E010E01AC0443608F04FC004E74C
:1051300010E0041B1109000F111F842F29830E9406
:10514000DE268595E82EFF24E7FCF094298137E1DF
:105150002302E00CF11C112468E070E0992031F08A
:105160008AED90E0AC014E195F097A01F601EE0F6D
:10517000FF1FEE0FFF1FEA5FFA4F0083E182C601B7
:10518000880F991F880F991FFC01EA5FFA4F2AE9DF
:105190002283992031F020E130E0F901E61BF70B82
:1051A000BF01FC01EA5FFA4F6430710514F48EE927
:1051B00009C06D3071052CF46A56628381E08383E7
:1051C0001CC08EEA861B8283138217C0C8010E940E
:1051D000822513C0992019F0F194E194F108F601A9
:1051E000EE0FFF1FEE0FFF1FEA5FFA4F80818A0D5F
:1051F000808381818E0D8183C2CF2296ECE00C9456
:10520000DA2F80E00E941A2B82FF0BC080910301ED
:10521000882339F080915B018F5F80935B0110924E
:10522000030180E00E941A2B82FD03C081E080937D
:10523000030180E00E941A2B85FF05C080910705BD
:105240008F5F8093070580910705893D18F088EDF1
:105250008093070580E00E941A2B84FF05C080918F
:10526000070581508093070580910705893018F460
:1052700089E08093070580E00E941A2B90FF25C0EB
:1052800080910401882309F1109204018091841017
:10529000803E60F080910605809383108091070521
:1052A0008093841088EC809385100FC080918710C4
:1052B000803E58F080910605809386108091070506
:1052C0008093871088EC8093881080E00E941A2BCE
:1052D00090FD03C081E0809304010895FC01EE0F6E
:1052E000FF1FE80FF91FED57FF4E20EE2183FC0151
:1052F000EE0FFF1FEE0FFF1FE25CFA4F21830895B0
:10530000CF93DF9325E0289FD001299FB00D112472
:10531000A757B04F2C91222309F450C01296CC917C
:105320001297FB01EE0FFF1FE60FF71FED57FF4E21
:10533000418124E0C202E0011124CA5FDA4F3981C1
:1053400020812A5F5881251B2C30C0F5242F231B78
:105350002B3FA4F1263094F511964C912091100F1B
:105360003091110F5AE0459F200D311D11243093CB
:10537000110F2093100F409101015091020142172B
:10538000530720F4309302012093010125E0289F68
:10539000F001299FF00D1124E757F04F8FEF818323
:1053A000A28184E0A802D0011124AA5FBA4F8BE643
:1053B00012968C931482CB010E946E29DF91CF91BB
:1053C000089525E0289FF001299FF00D1124E7574B
:1053D000F04F80818823F9F0948182819F3080F49E
:1053E0009F5F948324E08202F0011124EA5FFA4F68
:1053F0008BEA989F812D1124869585598283089583
:10540000118294E08902F0011124EA5FFA4F90EED4
:1054100091830E9442250895A0E0B0E0E2E1FAE223
:105420000C94C02F00E415E0C0E0D0E076EAF72E3F
:10543000CE010E946E29F801F08221960C5F1F4F69
:10544000C630D105A9F70E94EC2A40E051E060E0A7
:1054500070E08AE090E00E9423238DE480930805A9
:105460008AE08093060584E68093070581E090E05A
:105470000E94AB230E94A9240E944C2420E040916A
:10548000100F60E070E083E190E00E943B220E94F8
:1054900001290AE81FE0C0E0D0E0F80180819FEF19
:1054A000980F9E3F40F431978081882349F0CE01C8
:1054B0000E94FF2605C08F3F19F4CE010E94E1290A
:1054C00021960B5F1F4FC233D10539F704E810E175
:1054D000C3E8D0E155E8A52E50E1B52E6FE3C62E06
:1054E00065E0D62EE12CF12CF8018081803EF0F4AD
:1054F00088818850F501908192959F70890F8883EB
:10550000F80180818850F50190819F70890FF80122
:1055100080839881F60131979083F6018083983ECD
:1055200010F4803E18F0C7010E946E29FFEFEF1AB9
:10553000FF0A0D5F1F4F239683E0A80EB11CE4E025
:10554000CE0ED11CF6E0EF16F10471F60AE81FE06A
:10555000C0E0D0E0F801808181508E3F50F460E0DF
:1055600070E0CE010E94802961E070E0CE010E94CF
:10557000802921960B5F1F4FC233D10559F78091C7
:10558000920F833409F072CFE091900F84E0E8022B
:10559000F0011124EA5FFA4F408150E020E06BE116
:1055A00070E08AE090E00E946D22E091900F84E02C
:1055B000E802F0011124EA5FFA4F418150E020E057
:1055C0006BE170E084E190E00E946D224FCF809308
:1055D000AA0C9093AB0C0895E6E6F3E0A0EAB1E0E4
:1055E0006CE16D933197E9F7112408955091B40C53
:1055F000450F00C0992777272EE1629F080E191EDC
:10560000A0EAB1E0A00DB11D445E4C9311240895B1
:105610008093B40C08958093B20C9093B30C0895CA
:105620008091BA0C817008952091BA0C2E7F20933E
:10563000BA0C0895882329F48091C10C9091C20C72
:1056400008958091C50C9091C60C0895F999FECFEC
:1056500092BD81BD60BDF894FA9AF99A7894089544
:10566000F999FECF92BD81BDF894F89A80B57894EF
:10567000089599277727833008F00895E8E0F7E543
:10568000660F771FE60FF71FA591B491E4EFFEE0D8
:1056900026E0289FE00DF11DA183B2831124089517
:1056A00099277727E4EFFEE026E0289FE00DF11D23
:1056B0006E3F31F46091070F6E7F6093070F0BC050
:1056C0006F3F31F46091070F6E6F6093070F03C057
:1056D00079E5760F7583112408950000000000001D
:1056E00000000000000000000000000000000000BA
:1056F00000000000000000000000000000000000AA
:1057000080E08093F30E08952200240026002800F4
:105710002B002D0030003300360039003D004000E2
:10572000440048004C00510056005B0060006600D9
:105730006C00730079008100880090009900A2003D
:10574000AC00B600C100CC00D800E500F3000101B8
:10575000100121013201440157016C0181019801BE
:10576000B001CA01E501020221024102640288027D
:10577000AE02D7020303300361039403CB03050495
:1057800042048304C70410055D05AF0505066106E4
:10579000C206290796070908830805098E09200A09
:1057A000BA0A5D0B0A0CC10C840D510E2B0F12109E
:1057B00007110A121D1340147415BA161418831910
:1057C000071BA31C571E24200E22142439267F28D1
:1057D000E82A752D293006330F364539AD3C49404E
:1057E0001B442848734CFE50CF55EA5A51600C6652
:1057F0001D6C8B725A79928037885090E598FDA184
:105800009FABD3B5A3C00000000000000000000063
:105810000000000000000000000000000000000088
:105820000000000000000000000000000000000078
:105830000000000000000000000000000000000068
:105840000000000000000000000000000000000058
:105850000000000000000000000000000000000048
:105860000000000000000000000000000000000038
:105870000000000000000000000000000000000028
:105880000000000000000000000000000000000018
:105890000000000000000000000000000000000008
:1058A00000000000000000000000000000000000F8
:1058B00000000000000000000000000000000000E8
:1058C00000000000000000000000000000000000D8
:1058D00000000000000000000000000000000000C8
:1058E00000000000000000000000000000000000B8
:1058F00000000000000000000000000000000000A8
:10590000F9F8F9F5EBE1DDDEE0E2E4E5E6E5E4E215
:10591000DED9D2CAC1B7ACA299918A868381808030
:105920008182838586888A8C8D8F909293959697B5
:1059300098999A9B9B9C9D9D9D9E9E9E9F9F9F9F9D
:105940009F9F9F9E9E9E9D9D9D9C9B9B9A99989795
:1059500096959392908F8D8C8A888685838281809C
:10596000808183868A9199A2ACB7C1CAD2D9DEE27E
:10597000E4E5E6E5E4E2E0DEDDE1EBF5F9F8F90087
:105980000708070B151F2322201E1C1B1A1B1C1E99
:1059900022272E363F49545E676F767A7E7F7F7F5F
:1059A0007F7E7D7B7A7876747371706E6D6B6A69B9
:1059B00068676665656464636362626261616161B0
:1059C0006161616262626363636465656667686999
:1059D0006A6B6D6E7071737476787A7B7D7E7F7F73
:1059E0007F7F7E7A766F675E54493F362E27221E70
:1059F0001C1B1A1B1C1E2022231F150B0708070047
:105A00001F313D444E5354565A5F64696E74767923
:105A10007C7F7F7F7F7F7F7F7F7F7F7F7F7F7F7F99
:105A20007F7F7F7F7F7F7F7F7F7F7F7F7F7F7F7F86
:105A30007F7F7F7F7F7F7F7F7F7F7F7F7F7F7F7F76
:105A40007F7F7F7F7F7F7F7F7F7F7F7F7F7F7F7F66
:105A50007F7F7F7F7F7F7F7F7F7F7F7F7F7F7F7F56
:105A60007F7F7F7F7F7F7F7F7F7F7F7F7F7F7F7F46
:105A70007F7F7F7F7F7F7F7F7F7F7F7C7871684C98
:105A80002C1C120C0A0B0A05FDF3E9DFD4CAC0B7BF
:105A9000AEA69E97918B8685828080808080808054
:105AA00080808080808080808080808080808080F6
:105AB00080808080808080808080808080808080E6
:105AC00080808080808080808080808080808080D6
:105AD00080808080808080808080808080808080C6
:105AE00080808080808080808080808080808080B6
:105AF000808080808087919DACC4CBD4DDF2FAFA9F
:105B00007F7F7F7F7F7F7F7F7F7F7F7F7F7F7F7FA5
:105B10007F7F7F7F7F7F7F7F7F7F7F7F7F7F7F7F95
:105B20007F7F7F7F7F7F7F7F7F7F7F7F7F7F7F7F85
:105B30007F7F7F7F7F7F7F7F7F7F7F7F7F7F7F7F75
:105B40001D1D1D1D1D1D1D1D1D1D1D1D1D1D1E1E83
:105B50001E1E1D1D1D1D1D1D1D1D1D1D1D1C1C1C76
:105B60009F9F9F9FA0A0A0A1A1A1A1A1A1A1A1A130
:105B7000A1A1A0A0A0A0A0A0A0A0A0A0A0A0A0A023
:105B80005D5C5C5C5C5C5C5C5C5C5C5C5C5C5B5B56
:105B90005B5B5A5A5A5A5A5A5A5A5A5A5A59595966
:105BA000DCDCDCDCDDDDDDDEDEDEDEDEDEDEDEDE20
:105BB000DEDEDEDEDEDEDEDEDEDDDDDDDDDDDDDC0D
:105BC00080808080808080808080808080808080D5
:105BD00080808080808080808080808080808080C5
:105BE00080808080808080808080808080808080B5
:105BF00080808080808080808080808080808080A5
:105C00007F7F7F7F7F7F7F7F7F7F7F7F7F7F7F7FA4
:105C10007F7F7F7F7F7F7F7F7F7F7F7F7F7F7F7F94
:105C20007F7F7F7F7F7F7F7F7F7F7F7F7F7F7F7F84
:105C30007F7F7F7F7F7F7F7F7F7F7F7F7F7F7F7F74
:105C40008080808080808080808080808080808054
:105C50008080808080808080808080808080808044
:105C60008080808080808080808080808080808034
:105C70008080808080808080808080808080808024
:105C80008080808080808080808080808080808014
:105C90008080808080808080808080808080808004
:105CA00080808080808080808080808080808080F4
:105CB00080808080808080808080808080808080E4
:105CC00080808080808080808080808080808080D4
:105CD00080808080808080808080808080808080C4
:105CE00080808080808080808080808080808080B4
:105CF00080808080808080808080808080808080A4
:105D0000808182838485868788898A8B8C8D8E8F1B
:105D1000909192939495969798999A9B9C9D9E9F0B
:105D2000A0A1A2A3A4A5A6A7A8A9AAABACADAEAFFB
:105D3000B0B1B2B3B4B5B6B7B8B9BABBBCBDBEBFEB
:105D4000C0C1C2C3C4C5C6C7C8C9CACBCCCDCECFDB
:105D5000D0D1D2D3D4D5D6D7D8D9DADBDCDDDEDFCB
:105D6000E0E1E2E3E4E5E6E7E8E9EAEBECEDEEEFBB
:105D7000F0F1F2F3F4F5F6F7F8F9FAFBFCFDFEFFAB
:105D8000000102030405060708090A0B0C0D0E0F9B
:105D9000101112131415161718191A1B1C1D1E1F8B
:105DA000202122232425262728292A2B2C2D2E2F7B
:105DB000303132333435363738393A3B3C3D3E3F6B
:105DC000404142434445464748494A4B4C4D4E4F5B
:105DD000505152535455565758595A5B5C5D5E5F4B
:105DE000606162636465666768696A6B6C6D6E6F3B
:105DF000707172737475767778797A7B7C7D7E7F2B
:105E000089E091E00E940B2B89E091E00E94E72A53
:105E100080E00E94082BC1E081E090E00E94AB236B
:105E20000E94EC2A40E051E06AE070E08AE090E0F5
:105E30000E94232320E040915B016AE070E083E14F
:105E400090E00E943B2280915B01811103C044EFEE
:105E500050E002C048EE50E06BE070E08BE090E074
:105E60000E94232380E00E941A2B82FF0BC08091A6
:105E70000301882339F080915B018F5F80935B0180
:105E80001092030180E00E941A2B82FFC09303014D
:105E900080E00E941A2B83FFBFCF80915B01882393
:105EA00009F4BACF0E940C2A991B79E004C0991F0B
:105EB000961708F0961B881F7A95C9F78095089564
:105EC00087FB082E062687FD819567FD61950E9458
:105ED000542F0EF4919507FC81950895AA1BBB1BC6
:105EE00051E107C0AA1FBB1FA617B70710F0A61BDA
:105EF000B70B881F991F5A95A9F780959095BC01FB
:105F0000CD01089597FB072E16F4009407D077FD76
:105F100009D00E946E2F07FC05D03EF49095819524
:105F20009F4F0895709561957F4F0895A1E21A2EB5
:105F3000AA1BBB1BFD010DC0AA1FBB1FEE1FFF1F2D
:105F4000A217B307E407F50720F0A21BB30BE40B7D
:105F5000F50B661F771F881F991F1A9469F76095C4
:105F60007095809590959B01AC01BD01CF0108957E
:105F70002F923F924F925F926F927F928F929F9259
:105F8000AF92BF92CF92DF92EF92FF920F931F9347
:105F9000CF93DF93CDB7DEB7CA1BDB0B0FB6F894F8
:105FA000DEBF0FBECDBF09942A88398848885F8438
:105FB0006E847D848C849B84AA84B984C884DF80A9
:105FC000EE80FD800C811B81AA81B981CE0FD11D8D
:105FD0000FB6F894DEBF0FBECDBFED010895F89463
:025FE000FFCFF1
:105FE20001881301010405010000020304054100B8
:105FF200002B2D2F3100960006070809012C012ADB
:106002002C2E304158020C0D0E0F408A0216171822
:10601200190120031F20212201E8032425262741FC
:10602200E8031011121E00DC051A1B1C1D0D0102D3
:10603200030405060708090A0B0C0D0100030609F3
:106042000C101316181B1E212426292B2D2F313339
:106052003537383A3B3C3D3E3F3F4040000102026B
:0660620002FEFEFEFF003D
:00000001FF
